:100000000C942A000C944D2C1895000018950000B3
:10001000189500000C9456321895000018950000B1
:10002000189500001895000018950000189500001C
:10003000189500001895000018950000189500000C
:1000400018950000189500001895000018950000FC
:10005000189500008FE58DBFC0E4E0E14E2E88E0EA
:100060008EBFD8E0F8E05F2EEEEFF7E0A0E6B0E05C
:10007000A89584B7082E877F84BF88E1992781BD22
:1000800091BD88278D933197E9F70E94742D6624DE
:10009000E4E0F0E0A3EAB2E00E947533E5E0F0E0CE
:1000A000A6EAB2E00E947533E6E0F0E0A7EAB2E02B
:1000B0000E947533E7E0F0E0A8EAB2E00E947733EF
:1000C000E9E0F0E0AAEAB2E00E947533EAE0F0E08D
:1000D000ABEAB2E00E947733E0E0F0E0A0E6B0E007
:1000E0000E94753388EF8ABB8FE087BB83E084BBB7
:1000F00080EB81BB8FE482BB88E082BD85E085BD5B
:1001000089B7806489BF83E886B980EC87B98C9A07
:1001100083E38FBD81E08EBD789485B78C7F85BFEA
:100120008BB780648BBFA5E6B7E0EAEEF9E60E94E4
:10013000EF2F0E946A2EAEE6B7E0E4EFF9E60E94E8
:10014000EF2F0E94702E0E94062281E080934707C5
:10015000009147070D3118F011F00C94CD00E7E441
:10016000F7E0A190BB24EAE0F0E0AA0CBB1CEA0D8A
:10017000FB1DA7E4B7E0AD90BB24ABEAB2E0AA0C4C
:10018000BB1CAA0DBB1D0E947733A7E4B7E08C917E
:100190008F5F8C9310F40C94A80081E08093470744
:1001A000009147070E3E18F011F00C94FA00E7E4B6
:1001B000F7E0A190BB24E2E4F0E0AA0CBB1CAA0C7F
:1001C000BB1CEA0DFB1DA7E4B7E0AD90BB24A6E283
:1001D000B3E0AA0CBB1CAA0CBB1CAA0DBB1D94E06F
:1001E0000E947833A7E4B7E08C918F5F8C9310F472
:1001F0000C94D0000E9474220E94AC20C29A379ABC
:1002000007B1007E006007B90E94F52F082F192F53
:10021000003253E0150710F00C9426018FE711E02F
:100220000E94682DA1E6B0E00E944C2D8FEB11E0FA
:100230000E94682DA2E7B0E00E944C2DE4E0F0E0BF
:100240000E946B2D0C941E0A0C94560107B1007E7F
:10025000006007B90E94F52F082F192F043853E0CA
:10026000150710F00C9446018FE711E00E94682DED
:10027000A3E8B0E00E944C2D8FEB11E00E94682DA6
:10028000A2E7B0E00E944C2D0C9456018FE711E0DC
:100290000E94682DA4E9B0E00E944C2D8FEB11E084
:1002A0000E94682DA5EAB0E00E944C2D3798C298B4
:1002B000E2E0F0E00E946B2D80E08093490780E04F
:1002C00080935E07A2E9B2E00E94E631C198C0982F
:1002D0000E9474228FE711E00E94682DA6EBB0E027
:1002E0000E944C2D8FEB11E00E94682DA7ECB0E02E
:1002F0000E944C2D0E94AC200E949D208998A3EE64
:10030000B6E09C9194FF04C0819B10C09F7E9C939B
:1003100081990CC084E69F9399270E94522E9F9149
:10032000819904C090619C930E94CB0F8B98A3EE9F
:10033000B6E09C9193FF04C0839B10C0977F9C9371
:1003400083990CC084E69F9399270E94522E9F9117
:10035000839904C098609C930E94EA0F009149071A
:10036000013011F00C94CE018A98A3EEB6E09C9176
:1003700092FF04C0829B10C09B7F9C9382990CC00B
:1003800084E69F9399270E94522E9F91829904C0E0
:1003900094609C930C94A9020C949E02023011F07C
:1003A0000C94EC018A98A3EEB6E09C9192FF04C0F5
:1003B000829B10C09B7F9C9382990CC084E69F9384
:1003C00099270E94522E9F91829904C094609C9319
:1003D0000C9432030C949E02033011F00C940A0228
:1003E0008A98A3EEB6E09C9192FF04C0829B10C055
:1003F0009B7F9C9382990CC084E69F9399270E94CF
:10040000522E9F91829904C094609C930C94BB03DC
:100410000C949E02043011F00C9428028A98A3EEEA
:10042000B6E09C9192FF04C0829B10C09B7F9C937E
:1004300082990CC084E69F9399270E94522E9F9127
:10044000829904C094609C930C9411070C949E02B2
:10045000053011F00C9446028A98A3EEB6E09C9108
:1004600092FF04C0829B10C09B7F9C9382990CC01A
:1004700084E69F9399270E94522E9F91829904C0EF
:1004800094609C930C94A1080C949E02063011F089
:100490000C9464028A98A3EEB6E09C9192FF04C08B
:1004A000829B10C09B7F9C9382990CC084E69F9393
:1004B00099270E94522E9F91829904C094609C9328
:1004C0000C9444040C949E02073011F00C948202A8
:1004D0008A98A3EEB6E09C9192FF04C0829B10C064
:1004E0009B7F9C9382990CC084E69F9399270E94DE
:1004F000522E9F91829904C094609C930C94BD04E9
:100500000C949E02083011F00C949E028A98A3EE7F
:10051000B6E09C9192FF04C0829B10C09B7F9C938D
:1005200082990CC084E69F9399270E94522E9F9136
:10053000829904C094609C930C94A305A3EEB6E04A
:100540008C9186FB16F00C94A7020C94250A0C944F
:100550007E010E9474220E9484100E949D2089982E
:10056000A3EEB6E09C9194FF04C0819B10C09F7ED7
:100570009C9381990CC084E69F9399270E94522EE8
:100580009F91819904C090619C930E9484108B98E4
:10059000A3EEB6E09C9193FF04C0839B10C0977FAD
:1005A0009C9383990CC084E69F9399270E94522EB6
:1005B0009F91839904C098609C930E94A3108E9889
:1005C000A3EEB6E09C9191FF04C0869B10C09D7F76
:1005D0009C9386990CC084E69F9399270E94522E83
:1005E0009F91869904C092609C930E94D519889827
:1005F000A3EEB6E09C9190FF04C0809B10C09E7F4C
:100600009C9380990CC084E69F9399270E94522E58
:100610009F91809904C091609C930E9434178A989E
:10062000A3EEB6E09C9192FF04C0829B10C09B7F1A
:100630009C9382990CC084E69F9399270E94522E26
:100640009F91829904C094609C930C945C01A3EEEA
:10065000B6E08C9186FB16F00C9430030C94250ABE
:100660000C94AF020E9474220E941B130E949D20D2
:100670008998A3EEB6E09C9194FF04C0819B10C0C2
:100680009F7E9C9381990CC084E69F9399270E943A
:10069000522E9F91819904C090619C930E941B13DC
:1006A0008B98A3EEB6E09C9193FF04C0839B10C08F
:1006B000977F9C9383990CC084E69F9399270E940F
:1006C000522E9F91839904C098609C930E943A1384
:1006D0008E98A3EEB6E09C9191FF04C0869B10C05B
:1006E0009D7F9C9386990CC084E69F9399270E94D6
:1006F000522E9F91869904C092609C930E94D519B6
:100700008898A3EEB6E09C9190FF04C0809B10C037
:100710009E7F9C9380990CC084E69F9399270E94AA
:10072000522E9F91809904C091609C930E9434172F
:100730008A98A3EEB6E09C9192FF04C0829B10C001
:100740009B7F9C9382990CC084E69F9399270E947B
:10075000522E9F91829904C094609C930C945C01EA
:10076000A3EEB6E08C9186FB16F00C94B9030C94C2
:10077000250A0C9438030E9474220E946C140E9473
:100780009D208998A3EEB6E09C9194FF04C0819BC4
:1007900010C09F7E9C9381990CC084E69F939927FB
:1007A0000E94522E9F91819904C090619C930E9457
:1007B0006C148B98A3EEB6E09C9193FF04C0839BCE
:1007C00010C0977F9C9383990CC084E69F939927D0
:1007D0000E94522E9F91839904C098609C930E941E
:1007E0008B148E98A3EEB6E09C9191FF04C0869B7B
:1007F00010C09D7F9C9386990CC084E69F93992797
:100800000E94522E9F91869904C092609C930E94F0
:10081000D5198898A3EEB6E09C9190FF04C0809B08
:1008200010C09E7F9C9380990CC084E69F9399276B
:100830000E94522E9F91809904C091609C930E94C7
:1008400034178A98A3EEB6E09C9192FF04C0829B75
:1008500010C09B7F9C9382990CC084E69F9399273C
:100860000E94522E9F91829904C094609C930C9494
:100870005C01A3EEB6E08C9186FB16F00C9442046A
:100880000C94250A0C94C1030E9474220E94F9134F
:100890000E949D208998A3EEB6E09C9194FF04C02D
:1008A000819B10C09F7E9C9381990CC084E69F938E
:1008B00099270E94522E9F91819904C090619C9328
:1008C0000E94F9138B98A3EEB6E09C9193FF04C0AD
:1008D000839B10C0977F9C9383990CC084E69F9361
:1008E00099270E94522E9F91839904C098609C93EF
:1008F0000E94181400915E07033011F00C949A04C2
:100900008A98A3EEB6E09C9192FF04C0829B10C02F
:100910009B7F9C9382990CC084E69F9399270E94A9
:10092000522E9F91829904C094609C930C945C0118
:100930000C94B2048A98A3EEB6E09C9192FF04C096
:10094000829B10C09B7F9C9382990CC084E69F93EE
:1009500099270E94522E9F91829904C094609C9383
:100960000E94DA0EA3EEB6E08C9186FB16F00C9492
:10097000BB040C94250A0C944A040E947422EEE2F3
:10098000F9E60E94B331E7EAF2E0D080EE24FF24DA
:1009900000270E9471300E944931EDE0F0E0A1E4AF
:1009A000B7E00E945833E1E4F7E00E945230E2E3FE
:1009B000F9E60E94AA310E941831EDE0F0E0A1E4CE
:1009C000B7E00E945833E1E4F7E00E948834EDE09C
:1009D000F0E0A9EFB6E00E945833E1E4F7E00E94AE
:1009E000AE33EDE0F0E0ADEFB6E00E945833E1E465
:1009F000F7E00E94E233EDE0F0E0A1E0B7E00E9412
:100A000058330E94592D0E947D0C0E94AC200E94F8
:100A10009D20A2E9B2E00E94E6318998A3EEB6E0FB
:100A20009C9194FF04C0819B10C09F7E9C938199F0
:100A30000CC084E69F9399270E94522E9F91819922
:100A400004C090619C930E94E20B8B98A3EEB6E0E9
:100A50009C9193FF04C0839B10C0977F9C938399C4
:100A60000CC084E69F9399270E94522E9F918399F0
:100A700004C098609C930E94080C8E98A3EEB6E088
:100A80009C9191FF04C0869B10C09D7F9C9386998A
:100A90000CC084E69F9399270E94522E9F918699BD
:100AA00004C092609C930E94550C8898A3EEB6E017
:100AB0009C9190FF04C0809B10C09E7F9C93809966
:100AC0000CC084E69F9399270E94522E9F91809993
:100AD00004C091609C930E942E0C8A98A3EEB6E00D
:100AE0009C9192FF04C0829B10C09B7F9C93829933
:100AF0000CC084E69F9399270E94522E9F91829961
:100B000004C094609C930C945C01A2E9B2E00D9146
:100B10001C910B3350E0150718F011F00C9492055E
:100B20000C949805A2E9B2E00E94E6310E947D0C87
:100B3000A3EEB6E08C9186FB16F00C94A1050C9404
:100B4000250A0C940D050E9474220E9447150E94EC
:100B50009D208998A3EEB6E09C9194FF04C0819BF0
:100B600010C09F7E9C9381990CC084E69F93992727
:100B70000E94522E9F91819904C090619C930E9483
:100B800047158B98A3EEB6E09C9193FF04C0839B1E
:100B900010C0977F9C9383990CC084E69F939927FC
:100BA0000E94522E9F91839904C098609C930E944A
:100BB000661500915E07013011F00C94F9058A98D2
:100BC000A3EEB6E09C9192FF04C0829B10C09B7F75
:100BD0009C9382990CC084E69F9399270E94522E81
:100BE0009F91829904C094609C930C941E0A0C946B
:100BF000AB06023011F00C9417068A98A3EEB6E00B
:100C00009C9192FF04C0829B10C09B7F9C93829911
:100C10000CC084E69F9399270E94522E9F9182993F
:100C200004C094609C930C94B6060C94AB060330FD
:100C300011F00C9435068A98A3EEB6E09C9192FFD1
:100C400004C0829B10C09B7F9C9382990CC084E659
:100C50009F9399270E94522E9F91829904C094607D
:100C60009C930C946C0B0C94AB06043011F00C9418
:100C700053068A98A3EEB6E09C9192FF04C0829B33
:100C800010C09B7F9C9382990CC084E69F93992708
:100C90000E94522E9F91829904C094609C930C9460
:100CA0009A0B0C94AB06053011F00C9471068A98DF
:100CB000A3EEB6E09C9192FF04C0829B10C09B7F84
:100CC0009C9382990CC084E69F9399270E94522E90
:100CD0009F91829904C094609C930C94770A0C9421
:100CE000AB06063011F00C948F068A98A3EEB6E09E
:100CF0009C9192FF04C0829B10C09B7F9C93829921
:100D00000CC084E69F9399270E94522E9F9182994E
:100D100004C094609C930C94CC0B0C94AB060730ED
:100D200011F00C94AB068A98A3EEB6E09C9192FF6A
:100D300004C0829B10C09B7F9C9382990CC084E668
:100D40009F9399270E94522E9F91829904C094608C
:100D50009C930C945C01A3EEB6E08C9186FB16F09C
:100D60000C94B4060C94250A0C94A9058FEB11E0A1
:100D70000E94682DEEEFF9E60E94522D0E94AC20F1
:100D80000E94F215E6E3F9E60E94B331E9EEF6E0DF
:100D90000E944D300E941831EDE0F0E0ADE3B7E085
:100DA0000E945833EDE3F7E00E943734EDE0F0E0C5
:100DB0000E940F30A8E5B7E0EDE0FF270E9458330E
:100DC000E8E5F7E0AFE4B7E00E94B22F8FEB15E063
:100DD0000E94682DAFE4B7E00E944C2D8A98A3EEE4
:100DE000B6E09C9192FF04C0829B10C09B7F9C93B5
:100DF00082990CC084E69F9399270E94522E9F915E
:100E0000829904C094609C930C945C01A3EEB6E0BC
:100E10008C9186FB16F00C940F070C94250A0C9409
:100E2000C0060E9474220E944C218091E3068F77B5
:100E30008093E306A7EEB6E00E94E63185E080935A
:100E40004707009147070D3118F011F00C94460741
:100E5000A7EEB6E00D911C91A7E4B7E0AD90BB24DE
:100E6000ABEAB2E0AA0CBB1CAA0DBB1D4D915C9174
:100E7000040F151FA7EEB6E00D931C93A7E4B7E08F
:100E80008C918D5F8C9310F40C942107ADEAB2E045
:100E90008D919C91A2E9B2E08D939C93A2E9B2E07E
:100EA0000D911C91003050E0150718F011F00C94D2
:100EB0005B070C948D078FE711E00E94682DA8E076
:100EC000B3E00E944C2D8FEB13E00E94682DA8EF39
:100ED000B7E0E2E9F2E00E94FF320E944A2DA4EA64
:100EE000B1E00E944C2D8A98A3EEB6E09C9192FF4F
:100EF00004C0829B10C09B7F9C9382990CC084E6A7
:100F00009F9399270E94522E9F91829904C09460CA
:100F10009C930C945C010C944E0781E080934E07E7
:100F200000914E07093018F011F00C948908AEE4D6
:100F3000B7E00D91112743E050E00E94C22FA5E4D5
:100F4000B7E00D931C93A5E4B7E0AD90BC90AFEA79
:100F5000B2E0AA0CBB1CAA0DBB1D8D919C91A5EE05
:100F6000B6E08D939C938FEB11E00E94682DEEEF1D
:100F7000F9E60E94522DA5EEB6E00D911C910030CD
:100F800050E0150718F011F00C94C8070C94810874
:100F9000A5E4B7E0AD90BC90ABEAB2E0AA0CBB1CF4
:100FA000AA0DBB1D0D911C91003050E0150718F0E3
:100FB00011F00C94DD070C9477080091A302013026
:100FC00011F00C940C08AFEAB2E00D911C910030C6
:100FD00050E0150718F011F00C94F0070C940C0871
:100FE0000E94DA20AFEAB2E08D919C91A2E9B2E0D2
:100FF0008D939C938FE711E00E94682DA9E1B3E0E7
:101000000E944C2D0E94E72000914E070A3011F0FB
:101010000C940C080C9489080E94D320A5E4B7E036
:10102000AD90BC90ABEAB2E0AA0CBB1CAA0DBB1DF4
:101030008D919C91A2E9B2E08D939C938FE711E092
:101040000E94682DA5EBB1E00E944C2DA8EFB7E0FF
:10105000EEE4F7E00E940E330E944A2DA6ECB1E0C8
:101060000E944C2D0E94E72000914E070A3011F09B
:101070000C943C080C948908A5E4B7E0AD90BC90B2
:10108000ADEAB2E0AA0CBB1CAA0DBB1D8D919C91D0
:10109000A2E9B2E08D939C93A2E9B2E00D911C917C
:1010A000003050E0150718F011F00C9459080C941A
:1010B00077088FE711E00E94682DA5EBB1E00E9450
:1010C0004C2DA8EFB7E0EEE4F7E00E940E330E944B
:1010D0004A2DA7EDB1E00E944C2D0E94E72000911F
:1010E0004E070A3011F00C9477080C948908A5EE8D
:1010F000B6E00E94EA2CA7EEB6E00E94EA2C0C941F
:10110000BB07AEE4B7E08C918F5F8C9310F40C9426
:1011100090078FE711E00E94682DADE2B1E00E94D8
:101120004C2D8FEB11E00E94682DA8EEB1E00E94DB
:101130004C2D0E94AC20E4E0F0E00E946B2D0C945A
:10114000FA000E9474220E944C218091E3068F775E
:101150008093E30681E080935E07E2E6F7E00E9479
:10116000512FAAE4B7E00D931D9388278D938C939C
:10117000AAE4B7E00D911D912D913C9140E851E515
:1011800061E070E00E94CC2FAAE4B7E00D931D93BC
:101190002D933D934FEF5FEF6FEF7FEFAEE5B7E03D
:1011A000AD90BB24A6E2B3E0AA0CBB1CAA0CBB1CEE
:1011B000AA0DBB1D0D911D912D913C910E94EC3209
:1011C00080E014F009F081E08F9300915E070F3EFC
:1011D00081E008F080E09F918923882311F40C942A
:1011E000060AAAE4B7E00D911D912D913C91AEE560
:1011F000B7E0AD90BB24A6E2B3E0AA0CBB1CAA0CDE
:10120000BB1CAA0DBB1D4D915D916D917C910E94FF
:10121000E232A8E5B7E00D931D932D933D93009125
:10122000A302013011F00C943609AFEAB2E00D913F
:101230001C91003050E0150718F011F00C942209B1
:101240000C943609A8E5B7E00D911D912D913C91C4
:10125000AFEAB2E04D915C91662777270E94E732B2
:10126000A8E5B7E00D931D932D933D938FEB11E00F
:101270000E94682DA4EAB1E00E944C2DEEE5F7E053
:10128000A190BB24E6E2F3E0AA0CBB1CAA0CBB1C99
:10129000EA0DFB1DA8EFB7E00E94B22F0E944A2D75
:1012A0008FE711E00E94682DA5EBB1E00E944C2D64
:1012B0000E94612EAEE6B7E00E944C2D8A98A3EE04
:1012C000B6E09C9192FF04C0829B10C09B7F9C93D0
:1012D00082990CC084E69F9399270E94522E9F9179
:1012E000829904C094609C930C94FA00EFE5F7E0B7
:1012F0000E94792FA0E1B0E04D915D916D917C91BC
:10130000A8E5B7E00D911D912D913C910E94EC3222
:1013100011F00C9450090091A302013011F00C94CB
:10132000EF09AFEAB2E00D911C91003050E01507D3
:1013300018F011F00C949E090C94EF090E94DA2029
:10134000A8E5B7E00D911D912D913C91AFEAB2E077
:101350004D915C91662777270E94E232A8E5B7E0BD
:101360000D931D932D933D938FE711E00E94682DFF
:10137000A6ECB1E00E944C2D0E94612EAEE6B7E0D3
:101380000E944C2D8A98A3EEB6E09C9192FF04C077
:10139000829B10C09B7F9C9382990CC084E69F9394
:1013A00099270E94522E9F91829904C094609C9329
:1013B0000C94FA00EFE5F7E00E94792FA0E1B0E08D
:1013C0004D915D916D917C91A8E5B7E00D911D91D6
:1013D0002D913C910E94EC3211F00C94B4098FE7EE
:1013E00011E00E94682DA7EDB1E00E944C2D0E94F3
:1013F000612EAEE6B7E00E944C2D0E94DA20AEE5E9
:10140000B7E08C918F5F8C930C94CA088FE711E042
:101410000E94682DAEE3B1E00E944C2D8FEB11E0ED
:101420000E94682DA8EEB1E00E944C2D0E94AC20D5
:10143000E4E0F0E00E946B2D0C94FA000E944C2135
:101440008AE00E94CE2DDB98D398DB9B0C943C0A5B
:101450000E94592D8FE711E00E94682DA8EDB0E0A1
:101460000E944C2D8FEB15E00E94682D0E94612E8A
:10147000AEE6B7E00E944C2D8C988BB780648BBF92
:101480008091E30680648093E30687E0E4EFF1E077
:10149000A2E30E94F83185B7806B85BF8895A3EEE3
:1014A000B6E08C9186FB0EF4F0CF0E940622EFE5A9
:1014B000F7E00E943C2FA0E1B0E00D911D912D912D
:1014C0003C9141E050E060E070E00E94E232A8E52B
:1014D000B7E00D931D932D933D93E8E5F7E0AEE65D
:1014E000B7E00E94B22F0E94702E0C94FA008FEB8E
:1014F00011E00E94682DE0E1FAE60E94522DADE372
:10150000B2E00E944C2D0E94AC2081E080934707FE
:10151000009147070D3118F011F00C94AE0AE7E482
:10152000F7E0A190BB24EAE0F0E0AA0CBB1CEA0DB6
:10153000FB1DA7E4B7E0AD90BB24ABEAB2E0AA0C78
:10154000BB1CAA0DBB1D7BE70E946633A7E4B7E076
:101550008C918F5F8C9310F40C94880A8FEB11E0C0
:101560000E94682DE6E1FAE60E94522DADE3B2E05A
:101570000E944C2D80E08093480781E080934707CC
:10158000009147070E3E18F011F00C94120BE7E49F
:10159000F7E0A190BB24E2E4F0E0AA0CBB1CAA0C8B
:1015A000BB1CEA0DFB1DA7E4B7E0AD90BB24A6E28F
:1015B000B3E0AA0CBB1CAA0CBB1CAA0DBB1D94E07B
:1015C0007BE70E9467330091470748E10E947F3321
:1015D000AEE4B7E08C9300914E07003011F00C940C
:1015E0000A0BA8E4B7E08C91865F8C938FEB12E036
:1015F0000E94682DA8EFB7E0E8E4F7E00E940E3300
:101600000E944A2DECE1FAE60E94522DADE3B2E0D1
:101610000E944C2DA7E4B7E08C918F5F8C9310F45F
:101620000C94C00A0E94AC20E1E0F0E0A0EAB2E035
:101630007BE70E946433E2E0F0E0A1EAB2E07BE7FE
:101640000E946433E3E0F0E0A2EAB2E07BE70E94AC
:101650006433E4E0F0E0A3EAB2E07BE70E946433A5
:10166000E5E0F0E0A6EAB2E07BE70E946433E6E062
:10167000F0E0A7EAB2E07BE70E946433E7E0F0E045
:10168000A8EAB2E07BE70E946633E9E0F0E0AAEA6C
:10169000B2E07BE70E946433EAE0F0E0ABEAB2E05C
:1016A0007BE70E946633E0E0F0E0A0E6B0E07BE795
:1016B0000E9464338FEB11E00E94682DEEE1FAE6A0
:1016C0000E94522DADE3B2E00E944C2D84EF91E0D8
:1016D0000E94522E0C945C018FEB11E00E94682D49
:1016E000ABE1B2E00E944C2D0E94AC2081E08093DF
:1016F0004707009147070D3118F011F00C94940B37
:10170000A7E4B7E0AD90BB24ABEAB2E0AA0CBB1CE7
:10171000AA0DBB1D0E94E631A7E4B7E08C918F5F54
:101720008C9310F40C94790BE2E0F0E00E946B2DA6
:101730000C945C018FEB11E00E94682DACE2B2E0EA
:101740000E944C2D0E94AC2081E0809347070091BD
:1017500047070E3E18F011F00C94C60BA7E4B7E053
:10176000AD90BB24A6E2B3E0AA0CBB1CAA0CBB1C28
:10177000AA0DBB1DEAE3F9E60E94D631A7E4B7E063
:101780008C918F5F8C9310F40C94A70BE2E0F0E047
:101790000E946B2D0C945C018FE711E00E94682D74
:1017A000E4E2FAE60E94522D8FEB11E00E94682DD0
:1017B000E6E3FAE60E94522D0E949D200E948720B7
:1017C0000C945C01A0E3B0E00C9101FB0EF41FC08F
:1017D000A1EFB6E00E94E32CA1EFB6E00D911C91C1
:1017E0000F3E50E015071CF011F00C94F90B0C940F
:1017F000FD0BA1EFB6E00E94E6310E947D0C0E9435
:10180000AC2082E390E00E94522E0C94E20B0895EB
:10181000A0E3B0E00C9103FB0EF41FC0A1EFB6E013
:101820000E94EA2CA1EFB6E00D911C91003050E02F
:1018300015070CF402C00C94230C8FEE90E0A1EF7E
:10184000B6E08D939C930E947D0C0E94AC2082E3B5
:1018500090E00E94522E0C94080C0895A0E3B0E092
:101860000C9100FB81E00EF480E08F93A3EFB6E0D3
:101870000D911C910A3550E0150780E00CF481E0D1
:101880009F918923882311F40C94540CA3EFB6E0A4
:101890000E94E32C0E947D0C0E94AC2082E390E029
:1018A0000E94522E0C942E0C0895A0E3B0E00C91EF
:1018B00006FB81E00EF480E08F93A3EFB6E00D917C
:1018C0001C91063A5FEF150780E014F009F081E003
:1018D0009F918923882311F40C947C0CA3EFB6E02C
:1018E0000E94EA2C0E947D0C0E94AC2082E390E0D2
:1018F0000E94522E0C94550C0895E3EFF6E0D1901F
:10190000E0808FEFE7FE8827F82E082F0E947130C5
:101910000E94A730E2E3F9E60E94AA310E94183142
:10192000EDE0F0E0A1E4B7E00E945833E1E4F7E035
:101930000E948834EDE0F0E0A9E0B7E00E9458335F
:10194000E1E4F7E00E94AE33EDE0F0E0ADE0B7E0B7
:101950000E945833E1E4F7E00E94E233EDE0F0E06A
:10196000A1E1B7E00E945833EDE0F7E00E94523069
:10197000EDEFF6E00E944D300E941831EDE0F0E00E
:10198000A5E1B7E00E945833E9E0F7E00E94523049
:10199000E9EFF6E00E944D300E941831EDE0F0E0F2
:1019A000ADE1B7E00E9458330E94F215E1EFF6E096
:1019B000D190E0808FEFE7FE8827F82E082F0E9455
:1019C00071300E94A730E9EEF6E00E944D300E948F
:1019D0004931EDE0F0E0ADEEB6E00E945833EDEEB7
:1019E000F6E00E944D30EEE3F9E60E94B3310E942A
:1019F000BC3110F00C940E0DE2E4F9E60E94B33114
:101A0000EDEEF6E00E944D300E945831EDE0F0E03E
:101A1000ADEEB6E00E9458330C942E0DEDEEF6E0DC
:101A20000E944D30E6E4F9E60E94B3310E94BC31D9
:101A300018F011F00C941E0D0C942E0DE2E4F9E652
:101A40000E94B331EDEEF6E00E944D300E94493124
:101A5000EDE0F0E0ADEEB6E00E945833EDEEF6E0DA
:101A60000E945230EAE4F9E60E94AA310E9418313D
:101A7000EDE0F0E0A1E4B7E00E945833E1E4F7E0E4
:101A80000E94AE33EDE0F0E0A5E0B7E00E945833ED
:101A9000E5E0F7E00E945230E5E1F7E00E944D30CA
:101AA0000E941831EDE0F0E0A9E1B7E00E94583360
:101AB000E5E0F7E00E945230EDE1F7E00E944D30A2
:101AC0000E941831EDE0F0E0A1E2B7E00E94583347
:101AD000E9E1F7E00E945230EDE1F7E00E944D307D
:101AE0000E945831EDE0F0E0A5E2B7E00E945833E3
:101AF000E1E2F7E00E945230E5E1F7E00E944D306C
:101B00000E945831EDE0F0E0A9E2B7E00E945833BE
:101B1000E5E2F7E00E945230E9E2F7E00E944D3042
:101B20000E94C230EDE0F0E0A9E2B7E00E94583335
:101B3000E5E2F7E00E945230E9E2F7E00E944D3022
:101B40000E94C230EDE0F0E0A9E2B7E00E94583315
:101B5000E9E2F7E00E945230EDEFF6E00E944D30EE
:101B60000E941831EDE0F0E0ADE2B7E00E9458339A
:101B7000EDE0F7E00E945230EDE2F7E00E944D30D8
:101B80000E94C230EDE0F0E0ADE2B7E00E945833D1
:101B9000E1E0F7E00E945230E1E1F7E00E944D30D1
:101BA0000E94C230EDE0F0E0A1E3B7E00E945833BC
:101BB000E5E0F7E00E945230E1E3F7E00E944D30AB
:101BC0000E941831EDE0F0E0A1E3B7E00E94583345
:101BD000E1E3F7E00E945230EDE2F7E00E944D3081
:101BE0000E944931EDE0F0E0A1E4B7E00E945833F3
:101BF000E1E4F7E00E945230EEE4F9E60E94AA31F7
:101C00000E941831EDE0F0E0A1E4B7E00E94583303
:101C1000EBEAF2E0D190E0808FEFE7FE8827F82E24
:101C2000082F0E9471300E94A730E1E4F7E00E9483
:101C30004D300E945831EDE0F0E0A5EFB6E00E9493
:101C40005833E5EFF6E00E948F33EDE0F0E0A1E4D9
:101C5000B7E00E945833E5EFF6E00E943734EDE03C
:101C6000F0E00E940F30A5E4B7E0EE0C000FE7941F
:101C7000DD92EC92AFE4B7E0E5E4F7E00E940733D1
:101C8000E5E2F7E00E944D30E2E5F9E60E94B3316B
:101C90000E94BC3180E010F009F081E08F93E1E414
:101CA000F7E00E944D30E6E5F9E60E94B3310E946C
:101CB000BC3181E008F080E09F918923882311F4F2
:101CC0000C94740E8FE719E00E94682DEFE4F7E0A2
:101CD000A8EFB7E015E021E003E032E00E94033214
:101CE0000E944A2D0C947C0E8FE719E00E94682D0B
:101CF000A4EAB1E00E944C2DEDEEF6E00E943734EC
:101D0000EDE0F0E00E940F30A5E4B7E0EE0C000F2C
:101D1000E794DD92EC92AFE4B7E0E5E4F7E00E94EF
:101D200007338FE711E00E94682DEFE4F7E0A8EF9A
:101D3000B7E014E021E002E031E00E9403320E94AB
:101D40004A2DE8E4FAE60E94522DAFE4B7E0E1EF55
:101D5000F6E00E9407338FEB13E00E94682DEFE45A
:101D6000F7E0A8EFB7E013E0222702E031E00E949D
:101D700003320E944A2DE8E4FAE60E94522DAFE4B5
:101D8000B7E0E3EFF6E00E9407338FEB1BE00E9421
:101D9000682DEFE4F7E0A8EFB7E012E021E000E003
:101DA00033270E9403320E944A2DEAE4FAE60E9499
:101DB000522D08958FE711E00E94682DA7EDB1E044
:101DC0000E944C2D8FEB11E00E94682DA8EEB1E02F
:101DD0000E944C2D0E94AC200E949D200E948720D2
:101DE000C19A0091A302013011F00C94070F8FE704
:101DF00011E00E94682DA9EFB1E00E944C2D0E94D5
:101E0000AC200E949D200E9487200E94DA20009131
:101E10005E07013011F00C94620F8FE711E00E9411
:101E2000682DAAE0B2E00E944C2D0E94AC200E94D6
:101E30009D200E9487200E944C218FE711E00E9484
:101E4000682DABE1B2E00E944C2D8FEB11E00E94B7
:101E5000682DACE2B2E00E944C2D0E94AC20809133
:101E6000E3068F778093E3060E94D320A2E9B2E0D5
:101E70000E94E631A0E3B0E00C9102FB0EF016C028
:101E80008FE71BE00E94682DA8EFB7E0E2E9F2E0DF
:101E90000E94FF320E944A2DECE4FAE60E94522D85
:101EA00084E690E00E94522E0C943A0F8FE711E0E6
:101EB0000E94682DA4EAB1E00E944C2D0E94AC2043
:101EC0000C94BC0F023011F00C94BC0F8FE711E0A2
:101ED0000E94682DAFE4B1E00E944C2D8FEB11E021
:101EE0000E94682DADE3B2E00E944C2D0E94AC2010
:101EF0000E949D200E9487200E94592D8FE711E0AB
:101F00000E94682DAEE4B2E00E944C2D8FEB11E0F0
:101F10000E94682DABE1B2E00E944C2D0E94AC20E3
:101F20000E94D320A2E9B2E00E94E631A0E3B0E033
:101F30000C9102FB0EF418C08FEB1BE00E94682D81
:101F4000A8EFB7E0E2E9F2E00E94FF320E944A2DDA
:101F5000ECE4FAE60E94522D0E94AC2084E690E068
:101F60000E94522E0C94960F8FE711E00E94682D6C
:101F7000A5EBB1E00E944C2DC098C1988FEB11E009
:101F80000E94682DA9EEB0E00E944C2D0E94AC206A
:101F90000E949D200895A9E4B7E08C918F5F8C93F7
:101FA00000914907083080E010F009F081E08F933C
:101FB00000914907013081E008F080E09F91892B72
:101FC000882311F40C94E70F81E0809349070E9465
:101FD0000910089580914907815080934907009125
:101FE0004907013081E008F080E08F9300914907B4
:101FF000083080E010F009F081E09F91892B882360
:1020000011F40C94061088E0809349070E9409108F
:10201000089500914907013011F00C9419108FE7D1
:1020200011E00E94682DAAEFB0E00E944C2D0C94A4
:102030007910023011F00C9427108FE711E00E9404
:10204000682DABE0B1E00E944C2D0C947910033068
:1020500011F00C9435108FE711E00E94682DACE16F
:10206000B1E00E944C2D0C947910043011F00C94C6
:1020700043108FE711E00E94682DADE2B1E00E94AD
:102080004C2D0C947910053011F00C9451108FE701
:1020900011E00E94682DAEE3B1E00E944C2D0C943B
:1020A0007910063011F00C945F108FE711E00E9458
:1020B000682DAFE4B1E00E944C2D0C9479100730EC
:1020C00011F00C946D108FE711E00E94682DA0E6CE
:1020D000B1E00E944C2D0C947910083011F00C9452
:1020E00079108FE711E00E94682DA1E7B1E00E940E
:1020F0004C2D8FEB11E00E94682DA9EEB0E00E94FC
:102100004C2D0E94AC200895AEE5B7E08C918F5F16
:102110008C9300915E070C3080E010F009F081E0B4
:102120008F9300915E07013081E008F080E09F917D
:10213000892B882311F40C94A01081E080935E0712
:102140000E94C210089580915E07815080935E07BF
:1021500000915E07013081E008F080E08F930091EC
:102160005E070C3080E010F009F081E09F91892B30
:10217000882311F40C94BF108CE080935E070E94BA
:10218000C21008950E94592D00915E07013011F090
:102190000C94E2108FE711E00E94682DA4EAB1E0F0
:1021A0000E944C2D8FEB18E00E94682DA8EFB7E03D
:1021B000E2EAF2E00E940E330E944A2D0E94AC2017
:1021C0000C941A13023011F00C9419118FEF8093B4
:1021D000E2068FE711E00E94682DA5EBB1E00E94B6
:1021E0004C2D8FEB18E00E94682DA8EFB7E0E0EAD5
:1021F000F2E00E940E330E944A2D02E010E0A0EAB5
:10220000B2E04D9155270E94312DA6E5B7E00D9320
:102210001C93A6E5B7E00D911C9141E050E0041B32
:10222000150BA0E1B0E08D919C9199BD88BD0C94F7
:102230001A13033011F00C9450118FEF8093E206C3
:102240008FE711E00E94682DA6ECB1E00E944C2DB2
:102250008FEB18E00E94682DA8EFB7E0E1EAF2E00A
:102260000E940E330E944A2D02E010E0A1EAB2E083
:102270004D9155270E94312DA6E5B7E00D931C9393
:10228000A6E5B7E00D911C9141E050E0041B150B51
:10229000A0E1B0E08D919C9199BD88BD0C941A137A
:1022A000043011F00C946A118FE711E00E94682D40
:1022B000A7EDB1E00E944C2D8FEB15E00E94682D38
:1022C0000E94612EAEE6B7E00E944C2D0E94AC2029
:1022D0000C941A13053011F00C9484118FE711E05F
:1022E0000E94682DA8EEB1E00E944C2D8FEB15E006
:1022F0000E94682D0E94612EA5E6B7E00E944C2D39
:102300000E94AC200C941A13063011F00C94B011FA
:102310008FE711E00E94682DA9EFB1E00E944C2DDB
:102320000091A302003011F00C94A0118FEB11E08A
:102330000E94682DAAE0B2E00E944C2D0C94AC11D2
:10234000013011F00C94AC118FEB11E00E94682D5C
:10235000ABE1B2E00E944C2D0E94AC200C941A1309
:10236000073011F00C94DA11AFE4B7E0E6EAF2E0DE
:102370000E940E338FE711E00E94682DACE2B2E0BC
:102380000E944C2D8FEB14E00E94682DEFE4F7E0E3
:10239000A8EFB7E012E0222701E033270E940332C2
:1023A0000E944A2DADE3B2E00E944C2D0E94AC2069
:1023B0000C941A13083011F00C941012A7EAB2E032
:1023C0000D9111274AE550E0041B150BA5E4B7E079
:1023D0000D931C93AFE4B7E0E5E4F7E00E94073308
:1023E0008FE711E00E94682DAEE4B2E00E944C2D10
:1023F0008FEB17E00E94682DEFE4F7E0A8EFB7E05D
:1024000012E021E000E033270E9403320E944A2DAF
:10241000EAE4FAE60E94522D0E94AC200C941A13B2
:10242000093011F00C944612A8EAB2E00D911C910B
:1024300044EB50E0041B150BA5E4B7E00D931C938F
:10244000AFE4B7E0E5E4F7E00E9407338FE711E07F
:102450000E94682DAFE5B2E00E944C2D8FEB17E093
:102460000E94682DEFE4F7E0A8EFB7E012E021E06A
:1024700000E033270E9403320E944A2DEAE4FAE684
:102480000E94522D0E94AC200C941A130A3011F0B5
:102490000C947C12AAEAB2E00D9111274CE050E0B6
:1024A000041B150BA5E4B7E00D931C93AFE4B7E054
:1024B000E5E4F7E00E9407338FE711E00E94682D02
:1024C000A0E7B2E00E944C2D8FEB17E00E94682D30
:1024D000EFE4F7E0A8EFB7E012E021E000E03327F7
:1024E0000E9403320E944A2DE8E4FAE60E94522D2F
:1024F0000E94AC200C941A130B3011F00C94A6120D
:10250000AFE4B7E0EBEAF2E00E9407338FE711E0B7
:102510000E94682DA1E8B2E00E944C2D8FEB15E0DF
:102520000E94682DEFE4F7E0A8EFB7E0112721E063
:1025300003E032E00E9403320E944A2DEEE4FAE604
:102540000E94522D0E94AC200C941A130C3011F0F2
:102550000C941A1300916000003011F00C94C21218
:102560008FE711E00E94682DE2E5FAE60E94522D05
:102570008FEB11E00E94682DE4E6FAE60E94522DEE
:102580000C941813013011F00C94D8128FE711E05D
:102590000E94682DE6E7FAE60E94522D8FEB11E0CB
:1025A0000E94682DE8E8FAE60E94522D0C94181358
:1025B000023011F00C94EE128FE711E00E94682DAA
:1025C000EAE9FAE60E94522D8FEB11E00E94682D95
:1025D000ECEAFAE60E94522D0C941813033011F025
:1025E0000C9404138FE711E00E94682DEEEBFAE6DD
:1025F0000E94522D8FEB11E00E94682DE0EDFAE66B
:102600000E94522D0C941813043011F00C941813DE
:102610008FE711E00E94682DE2EEFAE60E94522D4B
:102620008FEB11E00E94682DE4EFFAE60E94522D34
:102630000E94AC200895AEE5B7E08C918F5F8C933B
:1026400000915E070D3180E010F009F081E08F937A
:1026500000915E07013081E008F080E09F91892BB6
:10266000882311F40C94371381E080935E070E9455
:102670005913089580915E07815080935E07009101
:102680005E07013081E008F080E08F9300915E07E3
:102690000D3180E010F009F081E09F91892B8823B3
:1026A00011F40C9456138DE180935E070E94591328
:1026B00008950E94592D00915E07033010F00C948C
:1026C00075138FE711E00E94682DAEE5B7E00D911C
:1026D000112741E150E00E94C22FA7EFB2E0A00F06
:1026E000B11F0E944C2D0C94AC1300915E0743E087
:1026F0000E947F33AEE4B7E00C938FE711E00E94B5
:10270000682DA4EAB1E00E944C2DA8EFB7E0EEE4FA
:10271000F7E00E940E330E944A2D00915E0743E0CD
:102720000E947F33AEE4B7E08C93AEE4B7E08C91C7
:102730008F5F8C938FE717E00E94682DAEE4B7E0BF
:102740000D9111274BE050E00E94C22FACEDB2E09A
:10275000A00FB11F0E944C2D00915E0743E00E9424
:102760007F33AEE4B7E08C9300914E07023081E0F6
:1027700009F080E08F9300915E07023080E010F056
:1027800009F081E09F918923882311F40C94DE13D2
:102790008FEB18E00E94682DA8EFB7E0EEE5F7E0B8
:1027A000A190BB24EBEAF2E0AA0CBB1CEA0DFB1DD6
:1027B0000E94FF320E944A2D0C94F6138FEB13E017
:1027C0000E94682DA8EFB7E0EEE5F7E0A190BB24EA
:1027D000EBEAF2E0AA0CBB1CEA0DFB1D0E94FF32E3
:1027E0000E944A2DA5EBB1E00E944C2D0E94AC2026
:1027F0000895AEE5B7E08C918F5F8C9300915E07F2
:10280000033080E010F009F081E08F9300915E07C3
:10281000013081E008F080E09F91892B882311F43A
:102820000C94151481E080935E070E94371408957C
:1028300080915E07815080935E0700915E070130B2
:1028400081E008F080E08F9300915E07033080E024
:1028500010F009F081E09F91892B882311F40C94EA
:10286000341483E080935E070E943714089500912A
:102870005E07013011F00C9447148FE711E00E94BD
:10288000682DA4EAB1E00E944C2D0C946114023032
:1028900011F00C9455148FE711E00E94682DA5EB00
:1028A000B1E00E944C2D0C946114033011F00C9493
:1028B00061148FE711E00E94682DA6ECB1E00E9440
:1028C0004C2D8FEB11E00E94682DA9EEB0E00E9424
:1028D0004C2D0E94AC200895AEE5B7E08C918F5F3F
:1028E0008C9300915E070E3E80E010F009F081E0CD
:1028F0008F9300915E07013081E008F080E09F91A6
:10290000892B882311F40C94881481E080935E074E
:102910000E94AA14089580915E07815080935E07FB
:1029200000915E07013081E008F080E08F93009114
:102930005E070E3E80E010F009F081E09F91892B48
:10294000882311F40C94A7148EEE80935E070E94E6
:10295000AA1408950E94592D8FE711E00E94682D56
:10296000A4EAB1E00E944C2DA8EFB7E0EEE5F7E055
:102970000E940E330E944A2D40E050E060E070E07B
:10298000AEE5B7E0AD90BB24A6E2B3E0AA0CBB1C59
:10299000AA0CBB1CAA0DBB1D0D911D912D913C9144
:1029A0000E94EC320CF402C00C94E0148FEB11E0A6
:1029B0000E94682DA5EBB1E00E944C2D0C944415AB
:1029C00040E851E561E070E0AEE5B7E0AD90BB24D2
:1029D000A6E2B3E0AA0CBB1CAA0CBB1CAA0DBB1D33
:1029E0000D911D912D913C910E94EC320CF402C08E
:1029F0000C9412158FEB15E00E94682DEEE5F7E0C0
:102A0000A190BB24E6E2F3E0AA0CBB1CAA0CBB1C01
:102A1000EA0DFB1DA8EFB7E00E94B22F0E944A2DDD
:102A20000C9444158FEB13E00E94682DEEE5F7E05F
:102A3000A190BB24E6E2F3E0AA0CBB1CAA0CBB1CD1
:102A4000EA0DFB1DA8EFB7E00E94B22F0E944A2DAD
:102A5000E6E0FBE60E94522DEEE5F7E0A190BB24F4
:102A6000E6E2F3E0AA0CBB1CAA0CBB1CEA0DFB1DA2
:102A70000E94382F002F112FA8EFB7E0E0E1F0E01F
:102A80000E94FF320E944A2D0E94AC200895AEE5BC
:102A9000B7E08C918F5F8C9300915E07073080E0E8
:102AA00010F009F081E08F9300915E07013081E022
:102AB00008F080E09F91892B882311F40C94631512
:102AC00081E080935E070E948515089580915E07DE
:102AD000815080935E0700915E07013081E008F02D
:102AE00080E08F9300915E07073080E010F009F0DE
:102AF00081E09F91892B882311F40C94821587E043
:102B000080935E070E948515089500915E0701304D
:102B100011F00C9495158FE711E00E94682DA4EA3E
:102B2000B1E00E944C2D0C94E715023011F00C948A
:102B3000A3158FE711E00E94682DA5EBB1E00E947C
:102B40004C2D0C94E715033011F00C94B1158FE760
:102B500011E00E94682DA6ECB1E00E944C2D0C946F
:102B6000E715043011F00C94BF158FE711E00E94B7
:102B7000682DA7EDB1E00E944C2D0C94E7150530AF
:102B800011F00C94CD158FE711E00E94682DA8EE8E
:102B9000B1E00E944C2D0C94E715063011F00C9416
:102BA000DB158FE711E00E94682DA9EFB1E00E94CC
:102BB0004C2D0C94E715073011F00C94E7158FE7B6
:102BC00011E00E94682DAAE0B2E00E944C2D8FEB2C
:102BD00011E00E94682DA9EEB0E00E944C2D0E94E9
:102BE000AC200895EFE5F7E00E943C2FA8E5B7E0A0
:102BF0000D931D932D933D93EAE5F9E60E94B331C1
:102C0000E8E5F7E00E944D300E9471300E94C2302A
:102C1000EDE0F0E0A5E3B7E00E945833EAEAF2E025
:102C2000D080EE24FF2400270E9471300E94A7303C
:102C3000E5E3F7E00E944D300E944931EDE0F0E01D
:102C4000A5E3B7E00E945833EEE5F9E60E94B33100
:102C5000E5E3F7E00E944D300E945831EDE0F0E0EE
:102C6000A5E3B7E00E945833E2E6F9E60E94B331EB
:102C7000E5E3F7E00E944D300E941831EDE0F0E00E
:102C8000A5E3B7E00E945833E2E6F7E00E94512F37
:102C9000A8E5B7E00D931D9388278D938C93E6E606
:102CA000F9E60E94B331E8E5F7E00E944D300E945A
:102CB00071300E941831EDE0F0E0A9E3B7E00E9426
:102CC0005833E9E3F7E00E945230E5E3F7E00E9471
:102CD0004D300E945831EDE0F0E0A5E3B7E00E94EE
:102CE0005833EAE6F9E60E94B331E5E3F7E00E94E3
:102CF0004D300E945831EDE0F0E0A5E3B7E00E94CE
:102D00005833EEE6F9E60E94B331E5E3F7E00E94BE
:102D10004D300E94C230EDE0F0E0A9E3B7E00E9440
:102D20005833E9E3F7E00E943734EDE0F0E00E9429
:102D30000F30A8E5B7E0EDE0FF270E945833E8E543
:102D4000F7E00E944D300E9471300E94A730E9E305
:102D5000F7E00E944D300E944931EDE0F0E0A5E33C
:102D6000B7E00E945833E2E4F9E60E94B331E5E3AC
:102D7000F7E00E944D300E941831EDE0F0E0A5E34D
:102D8000B7E00E945833E2E7F9E60E94B331E8EA7F
:102D9000F2E0D190E080FF2400270E9471300E9471
:102DA0004931EDE0F0E0A9E3B7E00E945833E6E7EF
:102DB000F9E60E94B331E9E3F7E00E944D300E944A
:102DC000C230EDE0F0E0A9E3B7E00E945833E9E358
:102DD000F7E00E945230E5E3F7E00E944D300E9498
:102DE0005831EDE0F0E0A9EEB6E00E945833E9EE8C
:102DF000F6E00E944D30EAE7F9E60E94B3310E9406
:102E0000BC3110F00C941617E2E4F9E60E94B331DD
:102E1000E9EEF6E00E944D300E945831EDE0F0E01E
:102E2000A9EEB6E00E9458330C943317E9EEF6E0B1
:102E30000E944D30E2E4F9E60E94B3310E94BC31B9
:102E400010F40C943317E2E4F9E60E94B331E9EE92
:102E5000F6E00E944D300E944931EDE0F0E0A9EE2D
:102E6000B6E00E945833089580E08093E406809194
:102E7000E30680628093E30600914907013011F078
:102E80000C94781800915E07013011F00C945A17D9
:102E9000A2EAB2E08C91A4E9B2E08D9388278D93E9
:102EA0008D938C93ACE9B2E0EEE7F9E60E94D6315F
:102EB0000C947618023011F00C947417A0EAB2E06A
:102EC0008C91A4E9B2E08D9388278D938D938C9398
:102ED000A1EAB2E08C91ACE9B2E08D9388278D93A2
:102EE0008D938C930C947618033011F00C948A1700
:102EF000A1EAB2E08C91A4E9B2E08D9388278D938A
:102F00008D938C93ACE9B2E0E2E8F9E60E94D63109
:102F10000C947618043011F00C94A817EFE5F7E044
:102F20000E943C2FA4E9B2E00D931D932D933D9395
:102F300080E0809347078091E30680628093E306F8
:102F4000ACE9B2E0E6E8F9E60E94D6310C947618D6
:102F5000053011F00C94BF17E2E6F7E00E94512F04
:102F6000A4E9B2E00D931D9388278D938C93ACE96F
:102F7000B2E0EAE8F9E60E94D6310C947618063001
:102F800011F00C94D517A3EAB2E08C91A4E9B2E059
:102F90008D9388278D938D938C93ACE9B2E0EEE806
:102FA000F9E60E94D6310C947618073011F00C9493
:102FB000EB17A6EAB2E08C91A4E9B2E08D938827E2
:102FC0008D938D938C93ACE9B2E0E2E9F9E60E942F
:102FD000D6310C947618083011F00C940918A7EA31
:102FE000B2E00C911127222733274AE550E060E038
:102FF00070E00E94E732A4E9B2E00D931D932D9397
:103000003D93ACE9B2E0E6E9F9E60E94D6310C94D2
:103010007618093011F00C942718A8EAB2E00D9147
:103020001C912227332744EB50E060E070E00E94BF
:10303000E732A4E9B2E00D931D932D933D93ACE9E3
:10304000B2E0EAE9F9E60E94D6310C9476180A302B
:1030500011F00C944518AAEAB2E00C91112722272E
:1030600033274CE050E060E070E00E94E732A4E9D2
:10307000B2E00D931D932D933D93ACE9B2E0EEE9E0
:10308000F9E60E94D6310C9476180B3011F00C94AE
:103090006218ABEAB2E08D919C91A4E9B2E08D9305
:1030A0009D9397FB26F48FEF8D938C9303C0882715
:1030B0008D938C93ACE9B2E0E2EAF9E60E94D63156
:1030C0000C9476180C3011F00C947618A0E6B0E051
:1030D0008C91A4E9B2E08D9388278D938D938C9386
:1030E000ACE9B2E0E6EAF9E60E94D6310C94551953
:1030F000023011F00C94A518AEE5B7E0AD90BB24FA
:10310000ABEAB2E0AA0CBB1CAA0DBB1D8D919C9131
:10311000A4E9B2E08D939D9388278D938C930091C1
:103120005E07023011F00C949D18ACE9B2E0EAEAB7
:10313000F9E60E94D6310C94A318ACE9B2E0EEEAAD
:10314000F9E60E94D6310C945519033011F00C9415
:103150005519AEE5B7E0AD90BB24A6E2B3E0AA0CEA
:10316000BB1CAA0CBB1CAA0DBB1D0D911D912D9162
:103170003C91A4E9B2E00D931D932D933C930091F3
:103180005E07013011F00C94D118EFE5F7E00E94D2
:103190003C2FA8E9B2E00D931D932D933D930C9421
:1031A000ED18AEE5B7E0AD90BB24A2E2B3E0AA0C07
:1031B000BB1CAA0CBB1CAA0DBB1D0D911D912D9112
:1031C0003C9149E050E060E070E00E94E232A8E902
:1031D000B2E00D931D932D933D93A8E9B2E04D917C
:1031E0005D916D917C91A4E9B2E00D911D912D91BD
:1031F0003C910E94EC320CF402C00C940B19A8E92B
:10320000B2E00D911D912D913C91A4E9B2E00D9396
:103210001D932D933C9300915E07033681E009F0E6
:1032200080E08F934FEF5FEF6FEF7FEFAEE5B7E09A
:10323000AD90BB24AAE2B3E0AA0CBB1CAA0CBB1C39
:10324000AA0DBB1D0D911D912D913C910E94EC3258
:1032500081E009F080E09F91892B882311F40C9480
:103260003919ACE9B2E0E2EBF9E60E94D6310C94F0
:103270005519AEE5B7E0AD90BB24AAE2B3E0AA0CC5
:10328000BB1CAA0CBB1CAA0DBB1D0D911D912D9141
:103290003C914AE050E060E070E00E94E732ACE927
:1032A000B2E00D931D932D933D93A0E3B0E00C91FC
:1032B00000FB81E00EF480E08F93ACE9B2E04D9129
:1032C0005D916D917C91A4E9B2E00D911D912D91DC
:1032D0003C910E94EC3280E00CF481E09F918923C4
:1032E000882311F40C94CF190E947321A4E9B2E051
:1032F0000D911D912D913C91A8E5B7E04D915D9107
:103300006D917C910E94E232A4E9B2E00D931D938D
:103310002D933D93ACE9B2E04D915D916D917C911F
:10332000A4E9B2E00D911D912D913C910E94EC32E7
:103330001CF011F00C949E190C94AA19ACE9B2E09F
:103340000D911D912D913C91A4E9B2E00D931D9337
:103350002D933C9300914907013011F00C94CB1947
:1033600000915E07043011F00C94CB19ACE9B2E087
:103370004D915D916D917C91A4E9B2E00D911D910B
:103380002D913C910E94EC3211F00C94CB19A4E9E0
:10339000B2E00E94E8310E94531C0C9455198091B0
:1033A000E3068F7D8093E306089580E08093E40632
:1033B0008091E30680628093E30600914907013023
:1033C00011F00C940F1B00915E07013011F00C946A
:1033D000F919A2EAB2E08C91A4E9B2E08D938827B2
:1033E0008D938D938C93A8E9B2E00E94E8310C9400
:1033F0000D1B023011F00C940D1AA0EAB2E08C9172
:10340000A4E9B2E08D9388278D938D938C93A8E9DE
:10341000B2E00E94E8310C940D1B033011F00C94C3
:10342000271AA1EAB2E08C91A4E9B2E08D93882733
:103430008D938D938C93A0EAB2E08C91A8E9B2E0D1
:103440008D9388278D938D938C930C940D1B043052
:1034500011F00C94451AEFE5F7E00E943C2FA4E927
:10346000B2E00D931D932D933D9380E08093470729
:103470008091E30680628093E306A8E9B2E0EAE384
:10348000F9E60E94D6310C940D1B053011F00C9416
:103490005A1AE2E6F7E00E94512FA4E9B2E00D9338
:1034A0001D9388278D938C93A8E9B2E00E94E831A0
:1034B0000C940D1B063011F00C946E1AA3EAB2E0C6
:1034C0008C91A4E9B2E08D9388278D938D938C9392
:1034D000A8E9B2E00E94E8310C940D1B073011F00E
:1034E0000C94841AA6EAB2E08C91A4E9B2E08D9320
:1034F00088278D938D938C93A8E9B2E0EEE8F9E6E6
:103500000E94D6310C940D1B083011F00C94A21AB5
:10351000A7EAB2E00C911127222733274AE550E0B1
:1035200060E070E00E94E732A4E9B2E00D931D93E1
:103530002D933D93A8E9B2E0E6EBF9E60E94D6317F
:103540000C940D1B093011F00C94C01AA8EAB2E0DB
:103550000D911C912227332744EB50E060E070E08E
:103560000E94E732A4E9B2E00D931D932D933D93A1
:10357000A8E9B2E0EAEBF9E60E94D6310C940D1B03
:103580000A3011F00C94DE1AAAEAB2E00C9111276D
:10359000222733274CE050E060E070E00E94E732E1
:1035A000A4E9B2E00D931D932D933D93A8E9B2E0F9
:1035B000EEEBF9E60E94D6310C940D1B0B3011F0A6
:1035C0000C94FB1AABEAB2E08D919C91A4E9B2E0B5
:1035D0008D939D9397FB26F48FEF8D938C9303C06F
:1035E00088278D938C93A8E9B2E0E2ECF9E60E947B
:1035F000D6310C940D1B0C3011F00C940D1BA0E671
:10360000B0E08C91A4E9B2E08D9388278D938D93DF
:103610008C93A8E9B2E00E94E8310C94B21B02300E
:1036200011F00C942C1BAEE5B7E0AD90BB24ABEAD7
:10363000B2E0AA0CBB1CAA0DBB1D8D919C91A4E904
:10364000B2E08D939D9388278D938C93A8E9B2E087
:103650000E94E8310C94B21B033011F00C94B21BA1
:10366000AEE5B7E0AD90BB24A6E2B3E0AA0CBB1C6C
:10367000AA0CBB1CAA0DBB1D0D911D912D913C9157
:10368000A4E9B2E00D931D932D933C9300915E0746
:10369000013081E009F080E08F934FEF5FEF6FEF33
:1036A0007FEFAEE5B7E0AD90BB24A2E2B3E0AA0C99
:1036B000BB1CAA0CBB1CAA0DBB1D0D911D912D910D
:1036C0003C910E94EC3281E009F080E09F91892BCF
:1036D000882311F40C94781BEFE5F7E00E943C2F4F
:1036E000A8E9B2E00D931D932D933D930C94B21B6A
:1036F000AEE5B7E0AD90BB24A2E2B3E0AA0CBB1CE0
:10370000AA0CBB1CAA0DBB1D0D911D912D913C91C6
:1037100049E050E060E070E00E94E232A8E9B2E0E7
:103720000D931D932D933D93A8E9B2E04D915D91CA
:103730006D917C91A4E9B2E00D911D912D913C9188
:103740000E94EC320CF402C00C94B21BA8E9B2E067
:103750000D911D912D913C91A4E9B2E00D931D9323
:103760002D933C93A0E3B0E00C9106FB81E00EF4B6
:1037700080E08F93A8E9B2E04D915D916D917C91CD
:10378000A4E9B2E00D911D912D913C910E94EC3283
:1037900080E014F009F081E09F918923882311F4DF
:1037A0000C944D1C0E947321A4E9B2E00D911D916F
:1037B0002D913C91A8E5B7E04D915D916D917C9183
:1037C0000E94E732A4E9B2E00D931D932D933D933F
:1037D00000914907033011F00C94081CA8E9B2E0ED
:1037E0004D915D916D917C91A4E9B2E00D911D9197
:1037F0002D913C910E94EC321CF011F00C94061CAF
:10380000A4E9B2E0EAE3F9E60E94D6310C94261C62
:10381000A8E9B2E04D915D916D917C91A4E9B2E08F
:103820000D911D912D913C910E94EC320CF402C03F
:103830000C94261CA8E9B2E00D911D912D913C91AC
:10384000A4E9B2E00D931D932D933C930091490799
:10385000013011F00C94491C00915E07043011F006
:103860000C94491CA8E9B2E04D915D916D917C9159
:10387000A4E9B2E00D911D912D913C910E94EC3292
:1038800011F00C94491CA4E9B2E0E6ECF9E60E94C0
:10389000D6310E94531C0C94B21B8091E3068F7D9D
:1038A0008093E30608958FEB11E00E94682DEEEF00
:1038B000F9E60E94522D00914907013011F00C9455
:1038C000DD1E00915E07013011F00C947D1C80918B
:1038D00094028093A2020E94892C8FEB18E00E9430
:1038E000682DA8EFB7E0E4E9F2E00E9402330E94FD
:1038F0004A2D0E94AC200C94DB1E023011F00C9477
:10390000B01C8FEF8093E206809194028093A00216
:1039100002E010E0A0EAB2E04D9155270E94312D5F
:10392000A6E5B7E00D931C93A6E5B7E00D911C91B9
:1039300041E050E0041B150BA0E1B0E08D919C919B
:1039400099BD88BD8FEB18E00E94682DA8EFB7E005
:10395000E4E9F2E00E9402330E944A2D0C94DB1E3F
:10396000033011F00C94E31C8FEF8093E2068091FA
:1039700094028093A10202E010E0A1EAB2E04D912E
:1039800055270E94312DA6E5B7E00D931C93A6E5BF
:10399000B7E00D911C9141E050E0041B150BA0E134
:1039A000B0E08D919C9199BD88BD8FEB18E00E948D
:1039B000682DA8EFB7E0E4E9F2E00E9402330E942C
:1039C0004A2D0C94DB1E043011F00C94141DA4E954
:1039D000B2E00D911D912D913C91A7E4B7E04C917F
:1039E0005527662777270E94E232A4E9B2E00D93BB
:1039F0001D932D933D9380E080934707E4E9F2E027
:103A0000AEE6B7E00E94B22F0E94702E8FEB15E059
:103A10000E94682D0E94612EAEE6B7E00E944C2DF8
:103A20000E94AC200C94DB1E053011F00C94401D5C
:103A3000A4E9B2E00D911D912D913C9140E851E532
:103A400061E070E00E94CC2FA8E5B7E00D931D93D4
:103A50002D933D93E8E5F7E0A5E6B7E00E94BA2F85
:103A60000E946A2E8FEB15E00E94682D0E94612E45
:103A7000A5E6B7E00E944C2D0E94AC200C94DB1E02
:103A8000063011F00C94761D809194028093A3026D
:103A900040E050E060E070E0A4E9B2E00D911D91DB
:103AA0002D913C910E94EC3211F00C94611D8FEB32
:103AB00011E00E94682DAAE0B2E00E944C2D0C9407
:103AC000721D41E050E060E070E00E94EC3211F0C5
:103AD0000C94721D8FEB11E00E94682DABE1B2E0F7
:103AE0000E944C2D0E94AC200C94DB1E073011F07C
:103AF0000C949C1D809194028093A602AFE4B7E0E1
:103B0000E4E9F2E00E9402338FEB14E00E94682D9A
:103B1000EFE4F7E0A8EFB7E012E0222701E0332757
:103B20000E9403320E944A2DADE3B2E00E944C2D68
:103B30000E94AC200C94DB1E083011F00C94C51DC3
:103B4000009194024AE5040FA7EAB2E00C93AFE4B7
:103B5000B7E0E4E9F2E00E9402338FEB17E00E9445
:103B6000682DEFE4F7E0A8EFB7E012E021E000E015
:103B700033270E9403320E944A2DEAE4FAE60E94AB
:103B8000522D0E94AC200C94DB1E093011F00C94D5
:103B9000F31DA4E9B2E00D911C9144EB50E0040F39
:103BA000151FA8EAB2E00D931C93AFE4B7E0E4E977
:103BB000F2E00E9402338FEB17E00E94682DEFE4E1
:103BC000F7E0A8EFB7E012E021E000E033270E9421
:103BD00003320E944A2DEAE4FAE60E94522D0E9426
:103BE000AC200C94DB1E0A3011F00C941C1E0091CA
:103BF00094024CE0040FAAEAB2E00C93AFE4B7E001
:103C0000E4E9F2E00E9402338FEB17E00E94682D96
:103C1000EFE4F7E0A8EFB7E012E021E000E033279F
:103C20000E9403320E944A2DE8E4FAE60E94522DD7
:103C30000E94AC200C94DB1E0B3011F00C94461E3D
:103C4000A4E9B2E08D919C91ABEAB2E08D939C9394
:103C5000AFE4B7E0E4E9F2E00E9402338FEB15E055
:103C60000E94682DEFE4F7E0A8EFB7E0112721E00C
:103C700003E032E00E9403320E944A2DEEE4FAE6AD
:103C80000E94522D0E94AC200C94DB1E0C3011F0CF
:103C90000C94DB1E809194028093600040E050E021
:103CA00060E070E0A4E9B2E00D911D912D913C918E
:103CB0000E94EC3211F00C946F1E8FE711E00E940D
:103CC000682DE2E5FAE60E94522D8FEB11E00E948A
:103CD000682DE4E6FAE60E94522D0C94D91E41E0CC
:103CE00050E060E070E00E94EC3211F00C948A1E0B
:103CF0008FE711E00E94682DE6E7FAE60E94522D58
:103D00008FEB11E00E94682DE8E8FAE60E94522D40
:103D10000C94D91E42E050E060E070E00E94EC326A
:103D200011F00C94A51E8FE711E00E94682DEAE9BE
:103D3000FAE60E94522D8FEB11E00E94682DECEA0A
:103D4000FAE60E94522D0C94D91E43E050E060E048
:103D500070E00E94EC3211F00C94C01E8FE711E06D
:103D60000E94682DEEEBFAE60E94522D8FEB11E0D7
:103D70000E94682DE0EDFAE60E94522D0C94D91EA7
:103D800044E050E060E070E00E94EC3211F00C94EE
:103D9000D91E8FE711E00E94682DE2EEFAE60E943C
:103DA000522D8FEB11E00E94682DE4EFFAE60E949D
:103DB000522D0E94AC200C94A11F023011F00C94E3
:103DC0002F1FA4E9B2E08D919C91AEE5B7E0AD90D4
:103DD000BB24ABEAB2E0AA0CBB1CAA0DBB1D8D93A1
:103DE0009C9300915E0743E00E947F33AEE4B7E00E
:103DF0008C9300914E07023081E009F080E08F93B0
:103E000000915E07023080E010F009F081E09F91A0
:103E10008923882311F40C941B1F8FEB18E00E9458
:103E2000682DA8EFB7E0E4E9F2E00E9402330E94B7
:103E30004A2D0C942B1F8FEB13E00E94682DA8EFE6
:103E4000B7E0E4E9F2E00E9402330E944A2DA5EBBC
:103E5000B1E00E944C2D0E94AC200C94A11F0330B5
:103E600011F00C94A11FA4E9B2E00D911D912D91C8
:103E70003C91AEE5B7E0AD90BB24A6E2B3E0AA0C5E
:103E8000BB1CAA0CBB1CAA0DBB1D0D931D932D932F
:103E90003C9340E050E060E070E0A4E9B2E00D91B6
:103EA0001D912D913C910E94EC320CF402C00C94B7
:103EB000631F8FEB11E00E94682DA5EBB1E00E941B
:103EC0004C2D0C949F1F40E851E561E070E0A4E99F
:103ED000B2E00D911D912D913C910E94EC320CF4B9
:103EE00002C00C94811F8FEB15E00E94682DE4E95D
:103EF000F2E0A8EFB7E00E94B22F0E944A2D0C9486
:103F00009F1F8FEB13E00E94682DE4E9F2E0A8EF19
:103F1000B7E00E94B22F0E944A2DE6E0FBE60E9425
:103F2000522DE4E9F2E00E94382F002F112FA8EF64
:103F3000B7E0E0E1F0E00E94FF320E944A2D0E94CB
:103F4000AC2084E690E00E94522E0895A3EEB6E0E5
:103F50008C9186FB16F00C94B91F8FEB15E00E9434
:103F6000682D0E94612EAEE6B7E00E944C2D0C94A5
:103F700086200091E2060F3F11F00C94C21F000052
:103F80000C9403200091E206053010F00C94E91F18
:103F9000A2EEB6E08C918F5F8C9302E010E0A1EA74
:103FA000B2E04D9155270E94312DACE5B7E00D935D
:103FB0001C93ACE5B7E00D911C9141E050E0041B6F
:103FC000150BA0E1B0E08D919C9199BD88BD0C943A
:103FD000032002E010E0A0EAB2E04D9155270E94D4
:103FE000312DACE5B7E00D931C93ACE5B7E00D9136
:103FF0001C9141E050E0041B150BA0E1B0E08D9155
:104000009C9199BD88BDA3EEB6E08C9187FB16F01C
:104010000C942E20A4EAB2E00D911C914CE350E0E8
:104020000E94172DACE5B7E04D935C93A6EAB2E091
:104030004D915527ACE5B7E00D911C91041715077C
:1040400010F40C942A208091E30680648093E306A8
:104050000C942E20A4EAB2E00E94E32C0091E40626
:10406000023310F00C943920A4EEB6E08C918F5FEF
:104070008C9300914907013011F00C945D20009160
:104080005E07043011F00C945B20A7E4B7E08C913C
:104090008F5F8C93A3EEB6E08C9185FB16F40C94A5
:1040A0005B208FEB15E00E94682D0E94612EAEE62A
:1040B000B7E00E944C2D0C948620043011F00C9433
:1040C0007420A2E9B2E00D911C91003050E0150778
:1040D00018F011F00C946E200C947220A2E9B2E05A
:1040E0000E94EA2C0C948620063011F00C947E205D
:1040F000A2E9B2E00E94E32C0C948620073011F074
:104100000C948620A2E9B2E00E94E32C0895A0E37B
:10411000B0E00C9102FB0EF00FC0A3EEB6E08C9164
:1041200086FB16F00C9496200C94250A84E690E009
:104130000E94522E0C9487200895A0E3B0E00C91C9
:1041400002FB0EF408C00E94AC2084E690E00E94BE
:10415000522E0C949D200895A4EAB2E00E94E6310C
:104160008091E30680688093E30680E08093E20616
:1041700002E010E0A1EAB2E04D9155270E94312DF6
:10418000A6E5B7E00D931C93A6E5B7E00D911C9151
:1041900041E050E0041B150BA0E1B0E08D919C9133
:1041A00099BD88BD0895C19A88EC90E00E94522E76
:1041B000C09A0895C19A88EC90E00E94522E80E047
:1041C000E8EFF4E2A8E30E94F831C1980895A2E96B
:1041D000B2E00D911C91003050E0150718F011F07D
:1041E0000C94F4200C9441218FEB11E00E94682D77
:1041F000A8EFB7E0E2E9F2E00E94FF320E944A2D08
:10420000EAE0FBE60E94522D8FEB17E00E94682D3A
:10421000A8EFB7E0E5EEF6E00E94FF320E944A2DDB
:10422000EEE0FBE60E94522D8FEB1CE00E94682D11
:104230008AE10E94C82DA8EFB7E0E7EEF6E00E9401
:10424000FF320E944A2DE2E1FBE60E94522D8A983D
:10425000A3EEB6E09C9192FF04C0829B10C09B7FAE
:104260009C9382990CC084E69F9399270E94522EBA
:104270009F91829904C094609C930E9444210C9465
:10428000E720C098C1980895A2E9B2E00E94E63103
:104290008AE080934E0708950E94AC208AEF90E058
:1042A0000E94522EA0E3B0E00C9102FB0EF418C065
:1042B0008FE711E00E94682DA2E8B1E00E944C2D2A
:1042C0008FEB11E00E94682DA3E9B1E00E944C2D14
:1042D0000E94AC2084E690E00E94522E0C94522161
:1042E0000E94592D08950091E406053010F00C94B9
:1042F0008121A8E5B7E0EEE8F9E60E94D6310C94FA
:1043000005220091E4060A3010F00C948F21A8E5F4
:10431000B7E0EAECF9E60E94D6310C940522009150
:10432000E4060F3010F00C949D21A8E5B7E0E2E818
:10433000F9E60E94D6310C9405220091E40604317E
:1043400010F00C94AB21A8E5B7E0EEECF9E60E9482
:10435000D6310C9405220091E406093110F00C943A
:10436000B921A8E5B7E0E2EDF9E60E94D6310C9458
:1043700005220091E4060E3110F00C94C721A8E547
:10438000B7E0E6EDF9E60E94D6310C9405220091E3
:10439000E406033210F00C94D521A8E5B7E0EAED6D
:1043A000F9E60E94D6310C9405220091E406083209
:1043B00010F00C94E321A8E5B7E0EEEDF9E60E94D9
:1043C000D6310C9405220091E4060D3210F00C94C5
:1043D000F121A8E5B7E0E2EEF9E60E94D6310C94AF
:1043E00005220091E406023310F00C94FF21A8E5A9
:1043F000B7E0E6EEF9E60E94D6310C940522A8E576
:10440000B7E0E6E8F9E60E94D63108958BB78F7BD6
:104410008BBFDB990C941C22D39ADB9A0E94742DDB
:1044200084E690E00E94522E88E00E94CE2D0E94E9
:10443000592D8CE00E94CE2D8C9AE1E0F0E0A0EAAC
:10444000B2E00E947533E2E0F0E0A1EAB2E00E943F
:104450007533E3E0F0E0A2EAB2E00E94753302E0D7
:1044600010E0A1EAB2E04D9155270E94312DA6E55A
:10447000B7E00D931C93A6E5B7E00D911C9141E0C8
:1044800050E0041B150BA0E1B0E08D919C9199BD0B
:1044900088BD0E94892C8FE711E00E94682DE4E11D
:1044A000FBE60E94522D8FEB11E00E94682DE6E2A0
:1044B000FBE60E94522D0E94AC20E2E0F0E00E9458
:1044C0006B2D82990C9473228FEF93E099BD88BD78
:1044D00087E08093A0028AE08093A1028AE0809323
:1044E000A2020E94AC20089500916000003011F0FB
:1044F0000C946E2400914907003011F00C941223A3
:10450000A1E6B0E0E8E3FBE60E94EF2FA2E7B0E00F
:10451000EAE4FBE60E94EF2FA3E8B0E0ECE5FBE65F
:104520000E94EF2FA4E9B0E0EEE6FBE60E94EF2F39
:10453000A5EAB0E0E0E8FBE60E94EF2FA6EBB0E0D2
:10454000E2E9FBE60E94EF2FA7ECB0E0E4EAFBE62D
:104550000E94EF2FA8EDB0E0E6EBFBE60E94EF2F04
:10456000A9EEB0E0E8ECFBE60E94EF2FAAEFB0E086
:10457000EAEDFBE60E94EF2FABE0B1E0ECEEFBE6EC
:104580000E94EF2FACE1B1E0EEEFFBE60E94EF2FCF
:10459000ADE2B1E0E0E1FCE60E94EF2FAEE3B1E076
:1045A000E2E2FCE60E94EF2FAFE4B1E0E4E3FCE6D8
:1045B0000E94EF2FA0E6B1E0E6E4FCE60E94EF2FB8
:1045C000A1E7B1E0E8E5FCE60E94EF2FA2E8B1E048
:1045D000EAE6FCE60E94EF2FA3E9B1E0ECE7FCE697
:1045E0000E94EF2FA8E0B3E0EEE8FCE60E94EF2F78
:1045F000A9E1B3E0E0EAFCE60E94EF2FA7EEB2E00B
:10460000E2EBFCE60E94EF2FA2EFB2E0EEEBFCE65D
:104610000E94EF2FADEFB2E0EAECFCE60E94EF2F34
:104620000C946C24013011F00C946C23A4EAB1E0DA
:10463000E6EDFCE60E94EF2FA5EBB1E0E8EEFCE62C
:104640000E94EF2FA6ECB1E0EAEFFCE60E94EF2F0C
:10465000A7EDB1E0ECE0FDE60E94EF2FA8EEB1E09F
:10466000EEE1FDE60E94EF2FA9EFB1E0E0E3FDE609
:104670000E94EF2FAAE0B2E0E2E4FDE60E94EF2FF5
:10468000ABE1B2E0E4E5FDE60E94EF2FACE2B2E080
:10469000E6E6FDE60E94EF2FADE3B2E0E8E7FDE6D7
:1046A0000E94EF2FAEE4B2E0E2E8FDE60E94EF2FB9
:1046B000AFE5B2E0E4E9FDE60E94EF2FA0E7B2E04B
:1046C000E6EAFDE60E94EF2FA1E8B2E0E8EBFDE6A6
:1046D0000E94EF2F0C946C24023011F00C947E2376
:1046E000A4EAB1E0EAECFDE60E94EF2FA5EBB1E011
:1046F000E0EDFDE60E94EF2F0C946C24033011F0E6
:104700000C949023A4EAB1E0EAEDFDE60E94EF2FBD
:10471000A5EBB1E0E8EEFDE60E94EF2F0C946C24CF
:10472000043011F00C94B423A4EAB1E0EAEFFDE602
:104730000E94EF2FA5EBB1E0EAECFDE60E94EF2F1F
:10474000A6ECB1E0E6E0FEE60E94EF2FA7EDB1E0B7
:10475000E2E1FEE60E94EF2FA8EEB1E0EEE1FEE618
:104760000E94EF2F0C946C24053011F00C94D82388
:10477000A4EAB1E0E0E3FEE60E94EF2FA5EBB1E092
:10478000E8E3FEE60E94EF2FA6ECB1E0E0E4FEE6EF
:104790000E94EF2FA7EDB1E0E8E4FEE60E94EF2FC4
:1047A000A8EEB1E0EEE1FEE60E94EF2F0C946C243F
:1047B000063011F00C942024A4EAB1E0E0E5FEE616
:1047C0000E94EF2FA5EBB1E0E2E6FEE60E94EF2F9C
:1047D000A6ECB1E0E4E7FEE60E94EF2FA7EDB1E022
:1047E000E6E8FEE60E94EF2FA8EEB1E0E8E9FEE67B
:1047F0000E94EF2FA9EFB1E0E0EAFCE60E94EF2F64
:10480000AAE0B2E0EAEAFEE60E94EF2FABE1B2E0F6
:10481000ECEBFEE60E94EF2FACE2B2E0E6ECFEE647
:104820000E94EF2FADE3B2E0E8EDFEE60E94EF2F2D
:10483000AEE4B2E0EAEEFEE60E94EF2F0C946C24A8
:10484000073011F00C942C24A4EAB1E0ECEFFEE662
:104850000E94EF2F0C946C24083011F00C946C24FF
:10486000A4EAB1E0E6E0FFE60E94EF2FA5EBB1E09D
:10487000E8E1FFE60E94EF2FA6ECB1E0EAE2FFE6F6
:104880000E94EF2FA7EDB1E0ECE3FFE60E94EF2FCF
:10489000A8EEB1E0EEE4FFE60E94EF2FA9EFB1E051
:1048A000E0E6FFE60E94EF2FAAE0B2E0E4E7FEE6D2
:1048B0000E94EF2FABE1B2E0E2E7FFE60E94EF2FAC
:1048C000ACE2B2E0E4E8FFE60E94EF2FADE3B2E035
:1048D000E6E9FFE60E94EF2F0C944C2C013011F01A
:1048E0000C94662600914907003011F00C940A25BB
:1048F000A1E6B0E0E4EAFFE60E94EF2FA2E7B0E015
:10490000E6EBFFE60E94EF2FA3E8B0E0E8ECFFE65D
:104910000E94EF2FA4E9B0E0EAEDFFE60E94EF2F3E
:10492000A5EAB0E0ECEEFFE60E94EF2FA6EBB0E0C8
:10493000EEEFFFE60E94EF2FA7ECB0E0E0E1F0E73A
:104940000E94EF2FA8EDB0E0E2E2F0E70E94EF2F27
:10495000A9EEB0E0E4E3F0E70E94EF2FAAEFB0E0A9
:10496000E6E4F0E70E94EF2FABE0B1E0E8E5F0E726
:104970000E94EF2FACE1B1E0EAE6F0E70E94EF2FF2
:10498000ADE2B1E0ECE7F0E70E94EF2FAEE3B1E07B
:10499000EEE8F0E70E94EF2FAFE4B1E0E0EAF0E7E5
:1049A0000E94EF2FA0E6B1E0E2EBF0E70E94EF2FCC
:1049B000A1E7B1E0E4ECF0E70E94EF2FA2E8B1E05C
:1049C000E6EDF0E70E94EF2FA3E9B1E0E8EEF0E7B3
:1049D0000E94EF2FA8E0B3E0EAEFF0E70E94EF2F8C
:1049E000A9E1B3E0ECE0F1E70E94EF2FA7EEB2E01F
:1049F000EEE1F1E70E94EF2FA2EFB2E0EAE2F1E789
:104A00000E94EF2FADEFB2E0E6E3F1E70E94EF2F57
:104A10000C946426013011F00C946425A4EAB1E0F2
:104A2000E2E4F1E70E94EF2FA5EBB1E0E4E5F1E766
:104A30000E94EF2FA6ECB1E0E6E6F1E70E94EF2F2F
:104A4000A7EDB1E0E8E7F1E70E94EF2FA8EEB1E0B3
:104A5000EAE8F1E70E94EF2FA9EFB1E0ECE9F1E716
:104A60000E94EF2FAAE0B2E0EEEAF1E70E94EF2FFA
:104A7000ABE1B2E0E0ECF1E70E94EF2FACE2B2E094
:104A8000E2EDF1E70E94EF2FADE3B2E0E4EEF1E7F3
:104A90000E94EF2FAEE4B2E0EEEEF1E70E94EF2FBE
:104AA000AFE5B2E0E0E0F2E70E94EF2FA0E7B2E06E
:104AB000E2E1F2E70E94EF2FA1E8B2E0E4E2F2E7E0
:104AC0000E94EF2F0C946426023011F00C9476258E
:104AD000A4EAB1E0E6E3F2E70E94EF2FA5EBB1E034
:104AE000ECE3F2E70E94EF2F0C946426033011F000
:104AF0000C948825A4EAB1E0E6E4F2E70E94EF2FE7
:104B0000A5EBB1E0E8EEFDE60E94EF2F0C946426E1
:104B1000043011F00C94AC25A4EAB1E0E4E5F2E72E
:104B20000E94EF2FA5EBB1E0E6E3F2E70E94EF2F42
:104B3000A6ECB1E0E0E6F2E70E94EF2FA7EDB1E0CE
:104B4000ECE6F2E70E94EF2FA8EEB1E0E8E7F2E72B
:104B50000E94EF2F0C946426053011F00C94D025A0
:104B6000A4EAB1E0EAE8F2E70E94EF2FA5EBB1E09A
:104B7000E2E9F2E70E94EF2FA6ECB1E0EAE9F2E702
:104B80000E94EF2FA7EDB1E0E2EAF2E70E94EF2FDB
:104B9000A8EEB1E0E8E7F2E70E94EF2F0C9464265C
:104BA000063011F00C941826A4EAB1E0EAEAF2E724
:104BB0000E94EF2FA5EBB1E0ECEBF2E70E94EF2FA4
:104BC000A6ECB1E0EEECF2E70E94EF2FA7EDB1E02A
:104BD000E0EEF2E70E94EF2FA8EEB1E0E2EFF2E79D
:104BE0000E94EF2FA9EFB1E0ECE0F1E70E94EF2F78
:104BF000AAE0B2E0E4E0F3E70E94EF2FABE1B2E01D
:104C0000E6E1F3E70E94EF2FACE2B2E0E0E2F3E787
:104C10000E94EF2FADE3B2E0E2E3F3E70E94EF2F53
:104C2000AEE4B2E0E4E4F3E70E94EF2F0C946426D4
:104C3000073011F00C942426A4EAB1E0ECEFFEE674
:104C40000E94EF2F0C946426083011F00C94642617
:104C5000A4EAB1E0E6E5F3E70E94EF2FA5EBB1E0AF
:104C6000E8E6F3E70E94EF2FA6ECB1E0EAE7F3E70E
:104C70000E94EF2FA7EDB1E0ECE8F3E70E94EF2FE1
:104C8000A8EEB1E0EEE9F3E70E94EF2FA9EFB1E063
:104C9000E0EBF3E70E94EF2FAAE0B2E0EEECF2E7E0
:104CA0000E94EF2FABE1B2E0E2ECF3E70E94EF2FBE
:104CB000ACE2B2E0E4EDF3E70E94EF2FADE3B2E047
:104CC000E6EEF3E70E94EF2F0C944C2C023011F02B
:104CD0000C945E2800914907003011F00C940227D3
:104CE000A1E6B0E0E4EFF3E70E94EF2FA2E7B0E027
:104CF000E6E0F4E70E94EF2FA3E8B0E0E8E1F4E794
:104D00000E94EF2FA4E9B0E0EAE2F4E70E94EF2F5F
:104D1000A5EAB0E0ECE3F4E70E94EF2FA6EBB0E0E9
:104D2000EEE4F4E70E94EF2FA7ECB0E0E0E6F4E752
:104D30000E94EF2FA8EDB0E0E2E7F4E70E94EF2F2A
:104D4000A9EEB0E0E4E8F4E70E94EF2FAAEFB0E0AC
:104D5000E6E9F4E70E94EF2FABE0B1E0E8EAF4E720
:104D60000E94EF2FACE1B1E0EAEBF4E70E94EF2FF5
:104D7000ADE2B1E0ECECF4E70E94EF2FAEE3B1E07E
:104D8000EEEDF4E70E94EF2FAFE4B1E0E0EFF4E7DF
:104D90000E94EF2FA0E6B1E0E2E0F5E70E94EF2FDE
:104DA000A1E7B1E0E4E1F5E70E94EF2FA2E8B1E06E
:104DB000E6E2F5E70E94EF2FA3E9B1E0E8E3F5E7CB
:104DC0000E94EF2FA8E0B3E0EAE4F5E70E94EF2F9E
:104DD000A9E1B3E0ECE5F5E70E94EF2FA7EEB2E022
:104DE000EEE6F5E70E94EF2FA2EFB2E0EAE2F1E78C
:104DF0000E94EF2FADEFB2E0E6E3F1E70E94EF2F64
:104E00000C945C28013011F00C945C27A4EAB1E00A
:104E1000EAE7F5E70E94EF2FA5EBB1E0ECE8F5E754
:104E20000E94EF2FA6ECB1E0EEE9F5E70E94EF2F2C
:104E3000A7EDB1E0E0EBF5E70E94EF2FA8EEB1E0BF
:104E4000E2ECF5E70E94EF2FA9EFB1E0E4EDF5E722
:104E50000E94EF2FAAE0B2E0E6EEF5E70E94EF2F06
:104E6000ABE1B2E0E8EFF5E70E94EF2FACE2B2E091
:104E7000EAE0F6E70E94EF2FADE3B2E0E4EEF1E7FF
:104E80000E94EF2FAEE4B2E0ECE1F6E70E94EF2FD4
:104E9000AFE5B2E0EEE2F6E70E94EF2FA0E7B2E066
:104EA000E0E4F6E70E94EF2FA1E8B2E0E4E2F2E7E7
:104EB0000E94EF2F0C945C28023011F00C946E27A6
:104EC000A4EAB1E0E6E3F2E70E94EF2FA5EBB1E040
:104ED000E2E5F6E70E94EF2F0C945C28033011F016
:104EE0000C948027A4EAB1E0ECE5F6E70E94EF2FEE
:104EF000A5EBB1E0E8EEFDE60E94EF2F0C945C28F4
:104F0000043011F00C94A427A4EAB1E0EAE6F6E735
:104F10000E94EF2FA5EBB1E0E6E3F2E70E94EF2F4E
:104F2000A6ECB1E0E6E7F6E70E94EF2FA7EDB1E0CF
:104F3000ECE6F2E70E94EF2FA8EEB1E0E2E8F6E738
:104F40000E94EF2F0C945C28053011F00C94C827B8
:104F5000A4EAB1E0E4E9F6E70E94EF2FA5EBB1E0A7
:104F6000ECE9F6E70E94EF2FA6ECB1E0E4EAF6E701
:104F70000E94EF2FA7EDB1E0ECEAF6E70E94EF2FD9
:104F8000A8EEB1E0E2E8F6E70E94EF2F0C945C286F
:104F9000063011F00C941028A4EAB1E0E4EBF6E737
:104FA0000E94EF2FA5EBB1E0E6ECF6E70E94EF2FB1
:104FB000A6ECB1E0E8EDF6E70E94EF2FA7EDB1E037
:104FC000EAEEF6E70E94EF2FA8EEB1E0E2EFF2E79B
:104FD0000E94EF2FA9EFB1E0ECE5F5E70E94EF2F7B
:104FE000AAE0B2E0ECEFF6E70E94EF2FABE1B2E00F
:104FF000EEE0F7E70E94EF2FACE2B2E0E8E1F7E77E
:105000000E94EF2FADE3B2E0EAE2F7E70E94EF2F54
:10501000AEE4B2E0EAE3F7E70E94EF2F0C945C28DD
:10502000073011F00C941C28A4EAB1E0ECEFFEE686
:105030000E94EF2F0C945C28083011F00C945C282F
:10504000A4EAB1E0EAE4F7E70E94EF2FA5EBB1E0B4
:10505000ECE5F7E70E94EF2FA6ECB1E0EEE6F7E70C
:105060000E94EF2FA7EDB1E0E0E8F7E70E94EF2FF5
:10507000A8EEB1E0E2E9F7E70E94EF2FA9EFB1E077
:10508000E4EAF7E70E94EF2FAAE0B2E0E8EDF6E7E6
:105090000E94EF2FABE1B2E0E6EBF7E70E94EF2FC3
:1050A000ACE2B2E0E8ECF7E70E94EF2FADE3B2E04C
:1050B000EAEDF7E70E94EF2F0C944C2C033011F02F
:1050C0000C94562A00914907003011F00C94FA28EC
:1050D000A1E6B0E0EAEEF7E70E94EF2FA2E7B0E02A
:1050E000ECEFF7E70E94EF2FA3E8B0E0EEE0F8E77F
:1050F0000E94EF2FA4E9B0E0E0E2F8E70E94EF2F72
:10510000A5EAB0E0E2E3F8E70E94EF2FA6EBB0E0FB
:10511000E4E4F8E70E94EF2FA7ECB0E0E6E5F8E75B
:105120000E94EF2FA8EDB0E0E2E2F0E70E94EF2F3F
:10513000A9EEB0E0E8E6F8E70E94EF2FAAEFB0E0B2
:10514000EAE7F8E70E94EF2FABE0B1E0ECE8F8E720
:105150000E94EF2FACE1B1E0EEE9F8E70E94EF2FFB
:10516000ADE2B1E0E0EBF8E70E94EF2FAEE3B1E093
:10517000E2ECF8E70E94EF2FAFE4B1E0E4EDF8E7EE
:105180000E94EF2FA0E6B1E0E2EBF0E70E94EF2FE4
:10519000A1E7B1E0E6EEF8E70E94EF2FA2E8B1E068
:1051A000E8EFF8E70E94EF2FA3E9B1E0EAE0F9E7C2
:1051B0000E94EF2FA8E0B3E0ECE1F9E70E94EF2FA7
:1051C000A9E1B3E0EEE2F9E70E94EF2FA7EEB2E02B
:1051D000E0E4F9E70E94EF2FA2EFB2E0ECE4F9E798
:1051E0000E94EF2FADEFB2E0E8E5F9E70E94EF2F64
:1051F0000C94542A013011F00C945429A4EAB1E023
:10520000E2E4F1E70E94EF2FA5EBB1E0E4E6F9E775
:105210000E94EF2FA6ECB1E0E6E7F9E70E94EF2F3E
:10522000A7EDB1E0E8E8F9E70E94EF2FA8EEB1E0C2
:10523000EAE9F9E70E94EF2FA9EFB1E0ECEAF9E71C
:105240000E94EF2FAAE0B2E0EEEBF9E70E94EF2F09
:10525000ABE1B2E0E4E5FDE60E94EF2FACE2B2E0A4
:10526000E2EDF1E70E94EF2FADE3B2E0E0EDF9E708
:105270000E94EF2FAEE4B2E0EAEDF9E70E94EF2FD3
:10528000AFE5B2E0ECEEF9E70E94EF2FA0E7B2E065
:10529000EEEFF9E70E94EF2FA1E8B2E0E0E1FAE7D4
:1052A0000E94EF2F0C94542A023011F00C946629BE
:1052B000A4EAB1E0E6E3F2E70E94EF2FA5EBB1E04C
:1052C000E2E2FAE70E94EF2F0C94542A033011F027
:1052D0000C947829A4EAB1E0ECE2FAE70E94EF2FFF
:1052E000A5EBB1E0E8EEFDE60E94EF2F0C94542A06
:1052F000043011F00C949C29A4EAB1E0EAE3FAE747
:105300000E94EF2FA5EBB1E0E6E3F2E70E94EF2F5A
:10531000A6ECB1E0E6E4FAE70E94EF2FA7EDB1E0DA
:10532000E2E5FAE70E94EF2FA8EEB1E0EEE5FAE73A
:105330000E94EF2F0C94542A053011F00C94C029D0
:10534000A4EAB1E0E0E7FAE70E94EF2FA5EBB1E0B5
:10535000E8E7FAE70E94EF2FA6ECB1E0E0E8FAE711
:105360000E94EF2FA7EDB1E0E8E8FAE70E94EF2FE7
:10537000A8EEB1E0EEE5FAE70E94EF2F0C94542A74
:10538000063011F00C94082AA4EAB1E0E0E9FAE74B
:105390000E94EF2FA5EBB1E0E2EAFAE70E94EF2FBF
:1053A000A6ECB1E0E4EBFAE70E94EF2FA7EDB1E045
:1053B000E6ECFAE70E94EF2FA8EEB1E0E2EFF2E7A9
:1053C0000E94EF2FA9EFB1E0EEE2F9E70E94EF2F84
:1053D000AAE0B2E0E8EDFAE70E94EF2FABE1B2E01D
:1053E000EAEEFAE70E94EF2FACE2B2E0E4EFFAE770
:1053F0000E94EF2FADE3B2E0E6E0FBE70E94EF2F63
:10540000AEE4B2E0E8E1FBE70E94EF2F0C94542AEF
:10541000073011F00C94142AA4EAB1E0ECEFFEE698
:105420000E94EF2F0C94542A083011F00C94542A47
:10543000A4EAB1E0EAE2FBE70E94EF2FA5EBB1E0BE
:10544000ECE3FBE70E94EF2FA6ECB1E0EEE4FBE714
:105450000E94EF2FA7EDB1E0E0E6FBE70E94EF2FFF
:10546000A8EEB1E0E2E7FBE70E94EF2FA9EFB1E081
:10547000E4E8FBE70E94EF2FAAE0B2E0E4EBFAE7F2
:105480000E94EF2FABE1B2E0E6E9FBE70E94EF2FCD
:10549000ACE2B2E0E8EAFBE70E94EF2FADE3B2E056
:1054A000EAEBFBE70E94EF2F0C944C2C043011F038
:1054B0000C944C2C00914907003011F00C94F22A06
:1054C000A1E6B0E0E8ECFBE70E94EF2FA2E7B0E036
:1054D000EAEDFBE70E94EF2FA3E8B0E0ECEEFBE77C
:1054E0000E94EF2FA4E9B0E0EEEFFBE70E94EF2F60
:1054F000A5EAB0E0E0E1FCE70E94EF2FA6EBB0E008
:10550000E2E2FCE70E94EF2FA7ECB0E0E4E3FCE767
:105510000E94EF2FA8EDB0E0E6E4FCE70E94EF2F39
:10552000A9EEB0E0E8E5FCE70E94EF2FAAEFB0E0BB
:10553000EAE6FCE70E94EF2FABE0B1E0EAE7FCE728
:105540000E94EF2FACE1B1E0ECE8FCE70E94EF2F06
:10555000ADE2B1E0EEE9FCE70E94EF2FAEE3B1E08F
:10556000E0EBFCE70E94EF2FAFE4B1E0E2ECFCE7F8
:105570000E94EF2FA0E6B1E0E2EBF0E70E94EF2FF0
:10558000A1E7B1E0E4EDFCE70E94EF2FA2E8B1E073
:10559000E6EEFCE70E94EF2FA3E9B1E0E8EFFCE7BD
:1055A0000E94EF2FA8E0B3E0EAE0FDE70E94EF2FB2
:1055B000A9E1B3E0ECE1FDE70E94EF2FA7EEB2E036
:1055C000EEE2FDE70E94EF2FA2EFB2E0EAE3FDE793
:1055D0000E94EF2FADEFB2E0E6E4FDE70E94EF2F6F
:1055E0000C944C2C013011F00C944C2BA4EAB1E03B
:1055F000E2E5FDE70E94EF2FA5EBB1E0E4E6FDE771
:105600000E94EF2FA6ECB1E0E6E7FDE70E94EF2F46
:10561000A7EDB1E0E8E8FDE70E94EF2FA8EEB1E0CA
:10562000EAE9FDE70E94EF2FA9EFB1E0ECEAFDE720
:105630000E94EF2FAAE0B2E0EEEBFDE70E94EF2F11
:10564000ABE1B2E0EEECFDE70E94EF2FACE2B2E09E
:10565000E2EDF1E70E94EF2FADE3B2E0E0EEFDE70F
:105660000E94EF2FAEE4B2E0EAEEFDE70E94EF2FDA
:10567000AFE5B2E0ECEFFDE70E94EF2FA0E7B2E06C
:10568000EEE0FEE70E94EF2FA1E8B2E0E0E2FEE7E5
:105690000E94EF2F0C944C2C023011F00C945E2BD6
:1056A000A4EAB1E0E6E3F2E70E94EF2FA5EBB1E058
:1056B000E2E3FEE70E94EF2F0C944C2C033011F034
:1056C0000C94702BA4EAB1E0ECE3FEE70E94EF2F0C
:1056D000A5EBB1E0E8EEFDE60E94EF2F0C944C2C18
:1056E000043011F00C94942BA4EAB1E0EAE4FEE754
:1056F0000E94EF2FA5EBB1E0E6E3F2E70E94EF2F67
:10570000A6ECB1E0E6E5FEE70E94EF2FA7EDB1E0E1
:10571000E2E6FEE70E94EF2FA8EEB1E0EEE6FEE73C
:105720000E94EF2F0C944C2C053011F00C94B82BE8
:10573000A4EAB1E0E0E8FEE70E94EF2FA5EBB1E0BC
:10574000E8E8FEE70E94EF2FA6ECB1E0E0E9FEE713
:105750000E94EF2FA7EDB1E0E8E8FAE70E94EF2FF3
:10576000A8EEB1E0EEE6FEE70E94EF2F0C944C2C81
:10577000063011F00C94002CA4EAB1E0E8E9FEE751
:105780000E94EF2FA5EBB1E0EAEAFEE70E94EF2FBF
:10579000A6ECB1E0ECEBFEE70E94EF2FA7EDB1E045
:1057A000EEECFEE70E94EF2FA8EEB1E0E2EFF2E7A9
:1057B0000E94EF2FA9EFB1E0ECE1FDE70E94EF2F8F
:1057C000AAE0B2E0E0EEFEE70E94EF2FABE1B2E02C
:1057D000E2EFFEE70E94EF2FACE2B2E0ECEFFEE773
:1057E0000E94EF2FADE3B2E0EEE0FFE70E94EF2F63
:1057F000AEE4B2E0EEE1FFE70E94EF2F0C944C2CF8
:10580000073011F00C940C2CA4EAB1E0ECEFFEE6AA
:105810000E94EF2F0C944C2C083011F00C944C2C5F
:10582000A4EAB1E0EEE2FFE70E94EF2FA5EBB1E0C2
:10583000E0E4FFE70E94EF2FA6ECB1E0E2E5FFE72E
:105840000E94EF2FA7EDB1E0E4E6FFE70E94EF2F03
:10585000A8EEB1E0E6E7FFE70E94EF2FA9EFB1E085
:10586000E8E8FFE70E94EF2FAAE0B2E0ECEBFEE7EA
:105870000E94EF2FABE1B2E0EAE9FFE70E94EF2FD1
:10588000ACE2B2E0ECEAFFE70E94EF2FADE3B2E05A
:10589000EEEBFFE70E94EF2F08950F921F922F92D9
:1058A0003F924F925F927F92AF92BF920F931F935E
:1058B0002F933F934F935F936F937F938F939F9318
:1058C000AF93BF93CF93DF93EF93FF938FB78F93F4
:1058D0008091E3068F7B8093E3068F918FBFFF91CA
:1058E000EF91DF91CF91BF91AF919F918F917F9178
:1058F0006F915F914F913F912F911F910F91BF90A9
:10590000AF907F905F904F903F902F901F900F909F
:105910001895A2EAB2E00D9111274FE050E0040F74
:10592000151FA6E5B7E00D931C93A6E5B7E00D9112
:105930001C914FE050E004231523A6E5B7E00D933A
:105940001C93A6E5B7E00D911C9140E750E0040FD1
:10595000151FA6E5B7E00D931C93A2EAB2E00C91E7
:105960001127222733274FE050E060E070E00E94CB
:10597000E232A8E5B7E00D931D932D933D9394E09B
:10598000A8E5B7E00E94FE2FA8E5B7E00D911D91B4
:105990002D913C9144E550E060E070E00E94E232DD
:1059A000A8E5B7E00D931D932D933D9389E2F6D0C2
:1059B00080915607F3D080915807F0D088E2EED05E
:1059C0000895F894FFCFED91FC91EF5FFF4FFC93AA
:1059D000EE930895ED91FC91E150F040FC93EE932D
:1059E000089509D00E94C22F00FC10D0089503D062
:1059F0001ED001F8F9CF0024E89457FF02C009D067
:105A0000689400F80BD010F80124089502D009D052
:105A10000895509540954F5F5F4F0895E89417FFA4
:105A20000895009510950F5F1F4F68940895352FC6
:105A3000242FE894452B11F468940895512F402F9A
:105A40000027112780E1440F551F001F111F021B63
:105A5000130B416018F4020F131F4E7F8A9599F7BC
:105A6000089514D081F0002E112E415050400ED0D8
:105A700009F408954F935F93402D512D0E94C22F3A
:105A80005F914F91F2CF01E0112708958827842B71
:105A9000852B0895A8EFB7E08D91882311F078D079
:105AA000FBCF08950E94A631802D11F071D0FACF5E
:105AB000089581E073D015D080E870C08FE7213061
:105AC00039F08FEB223021F08FE8233009F08FEC92
:105AD000810F0C94CE2D88EE93E0E4D03197D9F766
:105AE000089583E09927DEC08AEF90E00E94522E4D
:105AF000D49AD59AD69AD79AA19AA09AA89885E0CE
:105B000090E00E94522EA998DC98DD98DE9ADF9AE8
:105B1000A99AEF93FF93E5E1F0E00E94462EFF91F2
:105B2000EF91A998BCD0A99AEF93FF93E5E1F0E03B
:105B30000E94462EFF91EF91A998B1D0A99AEF93B8
:105B4000FF93E5E1F0E00E94462EFF91EF91A998C6
:105B5000A6D0DF98A99AEF93FF93E5E1F0E00E94C9
:105B6000462EFF91EF91A9989AD089E217D084E14F
:105B700015D085E513D08DE611D088E70FD088E2E7
:105B80000DD088E20BD08EE009D086E007D00895D2
:105B9000A89A829505D004D082D00895A898F9CF0C
:105BA000859510F4DF9A01C0DF98859510F4DE9A90
:105BB00001C0DE98859510F4DD9A01C0DD988595C9
:105BC00010F4DC9A01C0DC98A99AEF93FF93E5E109
:105BD000F0E00E94462EFF91EF91A998089500FCF5
:105BE00005D0089530D005D001F8F9CF37D03FD097
:105BF0000895842F952FA62FB72FE894452B462B79
:105C0000472B11F468940895402F512F622F732F62
:105C10000027112722273327F0E2440F551F661F64
:105C2000771F001F111F221F331F081B190B2A0B80
:105C30003B0B416028F4080F191F2A1F3B1F4E7FA2
:105C4000FA9559F708950024E89477FF02C006D02A
:105C5000689400F809D010F80124089512D04F5F1D
:105C60005F4F6F4F7F4F0895E89437FF0895009579
:105C70001095209530950F5F1F4F2F4F3F4F689421
:105C80000895409550956095709508953197F1F776
:105C90000895689462F80895E89462F8089581E0A0
:105CA00090E000C0EF93FF93EE27E82BE92B31F053
:105CB000EAEFF0E03197F1F70197D1F7FF91EF911B
:105CC0000895A5E6B7E0E2E6F7E00E94AE2E33972E
:105CD0000C948A2EE5E6F7E0A2E6B7E00E949C2E3F
:105CE000EEE6F7E0AFE5B7E00E94782EADE0BB2727
:105CF000868197810E944C320D93838194810E940A
:105D00004C320D93808191810E944C320D93089505
:105D1000EDE0FF2782810E9441328AE38D938181E9
:105D20000E9441328AE38D9380810E94413288270C
:105D30008C930895ADE0BB27808191810E944C3205
:105D40000D93838194810E944C320D9386819781BB
:105D50000E944C320D930895EDE0FF2780810E9450
:105D600041328EE28D9381810E9441328EE28D9389
:105D700082810E94413288278D93089593E0ADE09F
:105D800002C096E0AAE0B0E08FB7F89401910D93BD
:105D90009A95E1F78FBF08950191119145EB55E078
:105DA0000E94F72C440F440FF42E0F31150728F4EE
:105DB00081E0E82E0395D02E22C00C33150728F47D
:105DC00082E0E82E0E51D02E1AC00150150B4DE680
:105DD00051E00E94172DF40E7CE07A95872F9927C9
:105DE000E0E0FEE5A2E1BB270E94DE3102171307C7
:105DF000A0F37395E72E021B130B0395D02E089585
:105E000000001F003B005A0078009700B500D40046
:105E1000F300110130014E01019111912191308166
:105E200040E851E561E070E00E94F22D042F152F4B
:105E30000C94CE2EA3DF0E2D0A95802F02950032F2
:105E400020F01F2D137009F40395DA940D0D11271E
:105E50009927E4E6FEE5A8E1BB270E94E331080F9D
:105E6000111F0895000F1B2A384755647381909EB7
:105E70000E940C2F0C941B2F81DF0F2D11274CE358
:105E800055270E94F12C55270E0D151F4CE3222794
:105E90003327662777270E94CC2F0D0D131F231F52
:105EA00008956CDFDF92EF92FF920F2D11272227CA
:105EB00033274DE651E060E070E00E94CC2FFF9068
:105EC0004F2D4D5F469546955527662777270E94AB
:105ED000E232EF90DF900F931F932F933F930E9436
:105EE0001B2F222733277F916F915F914F910C9445
:105EF000E23247DFAF92BF92CF920E94522F40E82A
:105F000051E561E070E00E94CC2FFF90EF90DF90B0
:105F10000F931F932F933F930E943D2F7F916F917B
:105F20005F914F910C94E232019111912191308156
:105F300040E851E561E070E00E94F22D0C94A42F3E
:105F4000019111912191308140E15EE060E070E0CB
:105F50000E94F22DF42E4CE350E00E94F72CE42E28
:105F6000D02E0895AF93BF930E94942FBF91AF910D
:105F70000C94882EAF93BF930E940C2FBF91AF91CA
:105F80000C94AC2E0F92B801469F8001479F100DD4
:105F9000569F100D0F9008950F921F922F92C801D7
:105FA000D901489F80014A9F90014B9F202C499F17
:105FB000100D211D321D5A9F202C589F100D211DA0
:105FC000321D599F200D311D689F200D311D699F85
:105FD000300D789F300D2F901F900F9008950E94E4
:105FE000A6310D920020D9F70895369A3699FECF42
:105FF000369A3699FECF84B195B10895903071F0FC
:106000000D911D912D913C913695279517950795EA
:106010009A95D1F73C932E931E930E9308953DD0FD
:10602000992711278F2D880F80E8F82A802F881F45
:1060300008F41FEF41F08F57082F07FD04C000320E
:1060400040F08FEF01C08827982FD82EE82EF82E29
:1060500009C08FE1801B082FF694E794D794979599
:106060000A95D1F7112351F09095D094E094F094D3
:1060700081E0980F8827D81EE81EF81E0F2DFE2CF1
:10608000ED2CD92E0895D094E094F09491E0D90E9F
:106090009927E91EF91E10950895D190E190F1908D
:1060A0000191089521913191419151910895102FBD
:1060B00090E8FF0C001F0927990FF7941078652FBF
:1060C00090E8440F551F5927990F4795607800387D
:1060D0000895FF0C90E89027110F9795F794092FDA
:1060E0000895102FBD2CDE2CEF2CF02E11234AF436
:1060F000B094D094E094F0949FEFB91AD90AE90AC9
:10610000F90A0EE1FF2039F4FE2CED2CDB2CBB2428
:106110000850C2F76BC032F00A95BB0CDD1CEE1CB8
:10612000FF1CF9CF01D0D5CFB7FE089590E8B9167E
:1061300011F4D0FE08959FEFD91AE90AF90A09F47B
:1061400003950895DD92ED92FD920C930895502FE2
:106150002D2D3E2D4F2D612F08952DEC3CEC4CEC58
:106160005DE366270FC099DFF2DFDD24EE2490E8BF
:10617000F92E0FE307C096DF05C02227332740E240
:1061800051E46627552351F1002381F190DF71F12D
:106190001627005850580894050B18F407FD03C043
:1061A00025C007FD23C0469537952795F694E794BB
:1061B000D79422D0FF202AF0DD0CEE1CFF1C0150EA
:1061C00073F09D2D969548F0DD203AF4EE202AF4E8
:1061D00091E0D90E9927E91EF91E7BCF07C09FE7F2
:1061E000092FF92A9FEFD92EE92E0895DD24EE24F8
:1061F000FF240027112708959F929924AA24BB24E5
:1062000088E1D216E306F40628F0D21AE30AF40A6B
:10621000089401C08894991CAA1CBB1CDD0CEE1CC0
:10622000FF1C8A9571F7D92CEA2CFB2C9F900895BE
:106230003EDFE1F25038D1F216270058505808944A
:10624000051F12F418F4CBCF08F0D0CF0AD0FF20EE
:106250002AF0BB0CDD1CEE1CFF1C3BCF0F5FFBF1DB
:1062600038CF9F929924AA24BB24992788E1990CBE
:10627000AA1CBB1CDD1CEE1CFF1C30F4920EA31EDE
:10628000B41ED91EE91EF91E8A9589F79F900895BC
:1062900009DF0DDF503829F090E869270CC00AF0BB
:1062A00045D017CF5FE322273327442701C0FADE0A
:1062B000FEDE5038B1F3003899F3902F951B8BF325
:1062C00012F434D0FACF983118F02227332744271C
:1062D000983028F0232F342F44279850F9CF992352
:1062E00029F04695379527959A95D9F7912F9627B6
:1062F00042F014D0B0F6F794E794D7940F5F8BF682
:106300006ECF10D051F008F4BEDEFF2052F2DD0C4B
:10631000EE1CFF1C0150CBF762CF68CFD20EE31EFC
:10632000F41E0895D21AE30AF40A0895DF92EF9258
:10633000FF920F931F93D22EE32EF42E052F162FCC
:106340006F915F914F913F912F910895C89531962C
:1063500000200895FBDFD02CF9DFE02CF7DFF02CD4
:10636000F5DF002D0895F2DF202DF0DF302DEEDF78
:10637000402DECDF502D089507FB00680EF40F77D9
:1063800057FB50680EF45F7707FD02C057FF05C04A
:10639000D216E306F406050708952D153E054F05B0
:1063A0005007089591E005C092E003C094E001C059
:1063B00098E0CCDF0D929A95E1F70895880F991F28
:1063C000E80FF91FF1CFE80FF91FECCF82E001C011
:1063D00084E099279D938A95E9F7089591E08823B1
:1063E00021F08894991F8A95E9F7892F909508954F
:1063F000BB270E94EE319C9198279C933197F1F72F
:1064000098279C9308952E2E3F2E992781918D32A7
:1064100009F093958823D1F79A95E22DF32D112356
:1064200061F0091718F011F0101B01C0191B28F0BA
:1064300021F080E28D931A95E9F780818D3219F46D
:106440008D93319604C0222311F08BE28D930917AE
:1064500038F031F0091B21F080E38D930A95E9F7BC
:1064600081918D938823E1F7332351F0EA2FFB2F9D
:10647000319633958E9182933A95E1F78EE28C9323
:10648000089500278A3018F08A500395FBCF005DED
:106490000D93805D8D930895805390530027813034
:1064A00018F0065F8A95FBCF090F0895AF93BF934D
:1064B0000F939F938F938FB78F93AFE5B7E08C9136
:1064C00083958D938C3309F03DC088278E93119668
:1064D0008C9183958D938C3309F034C088278E93EB
:1064E00011968C9183958D93883161F588278E93D1
:1064F00011968C9183958D939C910EE1943089F047
:10650000963079F0993069F09B3059F00CE1923077
:1065100039F411969C911197937019F4039501C069
:106520000FE1801778F071F081E08E9311968C91D5
:1065300083958D938D3031F481E08E9311968C91FB
:1065400083958C938F918FBF8F919F910F91BF9166
:10655000AF910F921F922F923F924F925F927F9234
:10656000AF92BF920F931F932F933F934F935F93DD
:106570006F937F938F939F93AF93BF93CF93DF934B
:10658000EF93FF938FB78F930E94A61F8F918FBFBA
:10659000FF91EF91DF91CF91BF91AF919F918F913B
:1065A0007F916F915F914F913F912F911F910F912B
:1065B000BF90AF907F905F904F903F902F901F9033
:1065C0000F901895040F151F261F371F0895041BE1
:1065D000150B260B370B08950417150726073707E9
:1065E0000895000F111F221F331F08950095109565
:1065F000209530950F5F1F4F2F4F3F4F089501910A
:1066000010810EC001911191219130810BC0019137
:10661000108117FF05C03FEF2FEF04C00081112745
:106620002227332737FF03C0E1DF8DE28D93CF931D
:10663000DF93CF92DF92EF92AA24BB24CC24DD24F7
:10664000EE2440E2CAE0DD2755E093E38881890F1C
:1066500087FD9F7083FD907F891B89935A95A9F7C9
:10666000C0DFAA1CBB1CCC1CDD1CEE1C4A9551F7DC
:10667000E894EFE0FF2782910ED0EB30E0F71EF0B8
:1066800068948A2D0CD088278D93EF90DF90CF905F
:10669000DF91CF910895982F829501D0892F8F7027
:1066A000805D26F0803309F4089568948D930895F1
:1066B00094E081918D939A95E1F70895E199FECF49
:1066C000EEBBFFBB3196089591E001C092E07B37AD
:1066D00051F47FB7F894F2DF8D918DBBE29AE19A85
:1066E0009A95C9F77FBF7727089591E001C092E09E
:1066F000E5DFE09A8DB38D939A95D1F70895FF93D6
:10670000881BF9E0001FFA9511F4FF910895881F86
:10671000841B18F4840F8894F5CF0894F3CFBDDC64
:106720000F770895BADCC3DC0395AAF087E1DD0C8E
:10673000EE1CFF1C8A9589F00A95CAF7FF205AF0D3
:1067400000240D280E280F28002039F00A95DD0CB2
:10675000EE1CFF1CDAF70A95BCCC48CD9EDC85E028
:10676000C4D00F7723E839EF42E25EE361DDDBDF7F
:10677000E9DC139772D08A3F40F000688D3F18F42F
:1067800091DD80E803C0CED093DD88278483DFDCF1
:106790004FDDD8DC139729EA3EE64CE952EC48DDA0
:1067A00022E332E541E852E49CD022ED32EE4DE99D
:1067B00051EC97D020E93FEF4FE75FE379DD84812B
:1067C0000827A0C06ADC89E090D023E839EF42EACC
:1067D0005EE32EDDA8DF41D0902F907890870F7771
:1067E0008A3F50F08D3F28F49160908700685ADD11
:1067F00003C098D050685CDD8085807808271496A7
:10680000A1DC1797A4DC14DD9DDC13972DE334ED98
:106810004EE850EC66D025E13EED46E85FE348DD0A
:1068200096DC34963ADC3897ADDC14968BDC1797FF
:1068300034DC349724E536E748E450ECF9DC20E713
:1068400039ED43E550E434DD34962CDC3897F0DC48
:106850008085879508F488DC55C0802F9F2D991F6F
:10686000881F991F881F089518DC80E003C015DC7D
:10687000802F8078882321F0DF92EF92FF920F9390
:106880008F9315DC802F839512F4B0DC1BC08095AC
:106890008A95885E0AF415C088501AF40CD0D92263
:1068A00010C0DD2488501AF406D0E9220AC0EE2474
:1068B00002D0F92206C09FEF8770990F8A95EAF7F8
:1068C000089507DC8F918823D9F35F914F913F9111
:1068D0002F910F9351DD0F9199F390F323D05068CE
:1068E000E7CCE6DCDFDB3497A3CC0FB6F8944A9212
:1068F0005A92E42DF52DA42DB52D480E8827581E4B
:106900000FBE08950FB6F894599049900FBE0895A0
:10691000C4DB002331F02BED3FE049EC5FEBC8DC3A
:106920001ECF64CC5FE340E83327222708950000A0
:10693000B44203FA8E3C0000B443FFFFFFFF0000A7
:10694000F0C2000070430000F0424B77D63C0000DC
:106950002042CDCCCC3D00401C45000061450000EC
:106960004041B759803FDF92863DBF43D54000008C
:10697000C041000034430000C03F000000000F0091
:1069800000000A00000080510100AC8E00000100F0
:106990000000630000005A000000B40000000C007A
:1069A0000000E7030000040000001D0000000F27A6
:1069B00000007F33E101A6FFFFFF4DFFFFFFF4FF63
:1069C000FFFF19FCFFFF7F510100050000001E00C2
:1069D00000003C0000002C01000058020000100ED6
:1069E000000050460000A08C000030322E30382EBF
:1069F0003039000030303A30303A3030000020205A
:106A000020202020202020202020202020200000C6
:106A100020203025000020313025000025003130B5
:106A2000302500002056657273696F6E2020322E6B
:106A3000312E3420000030322E30382E32303039B2
:106A400020233746434100006800DF007300F42F25
:106A5000640020202020537072616368652020202C
:106A60002020000020202020646575747363682056
:106A7000202020200000202020206C616E6775619E
:106A8000676520202020000020202020656E676C94
:106A90006973682020202020000020202020206C06
:106AA000616E6775652020202020000020206C6525
:106AB000206672616E8761697320202000002020AB
:106AC000202020207461616C2020202020200000E4
:106AD0002020206E656465726C616E6473202020D6
:106AE000000020202020206C696E67756120202026
:106AF00020200000202020206974616C69616E6F85
:106B0000202020200000202B0000732000006E2099
:106B100000002000556E6976657273616C205469BF
:106B20006D6572200000627920506974202620541F
:106B3000542032303037000020426174746572692D
:106B400065206C65657220210000204269747465BF
:106B5000207765636873656C6E2000004261747411
:106B6000657269652073636877616368000020203F
:106B70004261747465726965204F4B2020200000CB
:106B800020207374617274652054696D65722020D1
:106B90000000202054696D65722062657265697419
:106BA000202000004D656E756520617573778468DF
:106BB0006C656E200000205374616E646279204D14
:106BC0006F647573202000004D656E7565206F64DD
:106BD000657220456E74657200002045696E73749D
:106BE000656C6C756E67656E202000002050726FBA
:106BF0006772616D6D7A656974656E200000202092
:106C0000205A65697470756E6B74652020200000D1
:106C10006175746F6D2E204175736C9473656E2071
:106C200000007A656974672E204175736C947365F2
:106C30006E200000206D616E2E204175736C947380
:106C4000656E20200000202020204B696E67726155
:106C5000746520202020000020202046756E6B7473
:106C6000696F6E656E2020200000202042697474D8
:106C700065205461737465202020000020206C6F13
:106C8000736C617373656E202120202000005761B2
:106C900072746520626973205374617274200000FD
:106CA0005370696567656C766F726175736C2E20C1
:106CB000000042656C69636874756E67000050611E
:106CC0007573652020202020000042696C64657285
:106CD00020202020000020204C4344204B6F6E7465
:106CE0007261737420200000204C43442048656C7E
:106CF0006C69676B6569742000006D61782E2048AF
:106D0000656C6C69676B656974200000205568725A
:106D10002065696E7374656C6C656E20000044615B
:106D200074756D2065696E7374656C6C656E0000BA
:106D3000202053564120616B746976203F2020202B
:106D400000002020202020206E65696E2020202059
:106D500020200000202020202020206A61202020E8
:106D600020202020000020506F7765722054696D2C
:106D7000656F757420200000204D696E7574656E16
:106D800000002067656F67722E2042726569746526
:106D900020200000202067656F67722E204C846ED3
:106DA000676520200000202020205A6569747A6FD2
:106DB0006E65202020200000204B6F7272656B747E
:106DC0007572776572742020000050726F67000042
:106DD0002053656B756E64656E00204175736C940D
:106DE00073657A65697420002020202020204E2FB2
:106DF000412020202020202000002053656B756E4C
:106E000064656E2000002042656C69636874756E6D
:106E1000670020506175736520202020200050728B
:106E20006F6772616D6D206265656E6465740000E8
:106E30002057617274652000204A65747A742000BE
:106E400020205356412020002020466F746F2000E0
:106E5000206D697420466573747374656C6C2020B2
:106E60000000206F686E6520466573747374656CEE
:106E70006C20000020696E732048617570746D6528
:106E80006E75652000002020466F6B757373696511
:106E900072656E20202000002020202020456E7486
:106EA00065722020202020200000204175736C9402
:106EB00073656E2053746172742000002042656C0B
:106EC0006963687465002053746F70206D69742065
:106ED000456E746572200000456E74657220756E93
:106EE000642068616C74656E0000204175666E6197
:106EF000686D65206C847566742000002020204E2B
:106F00002F41202000002020417573736368616C5D
:106F100074656E2020200000202020537465726E5E
:106F20007A65697420202020000050726F67722EED
:106F3000206C94736368656E203F00005A65697425
:106F4000702E206C94736368656E203F0000576557
:106F50007274652073706569636865726E200000E5
:106F60002020496E666F726D6174696F6E202020FB
:106F7000000050726F67722E2067656C94736368AF
:106F8000742000005A656974702E2067656C9473D4
:106F900063687420000020676573706569636865C5
:106FA0007274200020626174746572696520646582
:106FB00061642021000020706C656173652072653A
:106FC000706C616365200000206261747465726991
:106FD00065207765616B2020000020626174746514
:106FE0007269652077656C6C2020000020696E69ED
:106FF00074696174652074696D65722000002020D9
:1070000074696D65722072656164792020200000CA
:10701000202073656C656374206D656E752020207B
:10702000000020207374616E646279206D6F646566
:1070300020200000206D656E7565206F7220656EE2
:10704000746572200000202061646A7573746D6538
:107050006E747320202000002070726F6772616D63
:107060002074696D657320200000202074696D65AF
:1070700020706F696E747320202000002061757489
:107080006F6D2E2072656C65617365200000202095
:1070900074696D652072656C656173652020000000
:1070A00020206D616E2E2072656C656173652020F5
:1070B0000000202020206B696E67726174652020BB
:1070C0002020000020202066756E6374696F6E7347
:1070D00020202020000020706C656173652072659F
:1070E0006C65617365200000202020206275747437
:1070F0006F6E202120202020000077616974696E66
:107100006720746F2073746172740000206D69725F
:10711000726F72206C6F636B757020200000657851
:10712000706F737572652020000070617573652043
:10713000202020200000696D6167657320202020D9
:10714000000020204C434420636F6E74726173749E
:1071500020200000204C4344206272696768746EEE
:107160006573732000006D61782E20627269676814
:10717000746E6573732000002020202073657420D6
:1071800074696D6520202020000020202020736578
:1071900074206461746520202020000020204D4C64
:1071A0005520616374697665203F2020000020200F
:1071B00020202020206E6F20202020202020000072
:1071C00020202020202079657320202020202020CE
:1071D000000020706F7765722074696D656F75743B
:1071E00020200000206D696E75746573000067656E
:1071F0006F67722E206C617469747564652000007D
:1072000067656F67722E206C6F6E67697475646551
:10721000000020202074696D65207A6F6E65202043
:1072200020200000202020636F7272656374696FF4
:107230006E202020000070726F670000207365636D
:107240006F6E647320007472696767657220746979
:107250006D652000207365636F6E647320200000ED
:10726000206578706F7375726520200020706175DD
:10727000736520202020200070726F6772616D207E
:1072800066696E69736865640000202077616974BF
:10729000200020206E6F7720200020204D4C5520AC
:1072A0002000202073686F74200020202020206C94
:1072B0006F636B65642020202020000020202020A8
:1072C000756E6C6F636B65642020202000002020A9
:1072D000746F206D61696E206D656E7520200000F1
:1072E000202020666F63757373696E6720202020ED
:1072F00000002020202020656E7465722020202050
:10730000202000002073746172742072656C6561C6
:10731000736520200000206578706F73696E6700C8
:1073200020656E74657220746F2073746F702020F6
:10733000000020656E74657220616E6420686F6C59
:10734000642000002020202072756E6E696E672018
:10735000202020200000202020706F776572206F91
:107360006666202020200000202020207374617297
:1073700074696D6520202020000064656C6574656B
:107380002070726F6772616D203F00002064656C31
:107390006574652074696D6573203F20000073611A
:1073A000766520706172616D65746572732000008E
:1073B0002020696E666F726D6174696F6E20202087
:1073C000000070726F6772616D732064656C657424
:1073D000656400002074696D65732064656C657474
:1073E00065642020000020736176656420202020E1
:1073F00020202000202070696C65208520706C6141
:1074000074202020000020206368616E6765722070
:107410007376702020200000202070696C65206643
:107420006169626C652020200000202020207069A6
:107430006C65204F4B202020202000002064826DAE
:1074400061727265722074696D657220000020207F
:107450002074696D6572207072887420202000008D
:10746000202063686F69736972206D656E752020D6
:10747000000020206D6F646520617474656E746512
:1074800020200000206D656E7565206F7520656E8B
:10749000746572200000202020207282676C616772
:1074A000657320202020000070726F6772616D6D1F
:1074B000652074656D7073200000207074732074F3
:1074C000656D706F72656C73202000006482636C60
:1074D000656E63682E206175746F6D2E0000686F95
:1074E00072206482636C656E6368656D2E20000097
:1074F0006482636C656E6368656D2E206D616E7568
:10750000000020202072826672616374696F6E20B1
:1075100020200000202020666F6E6374696F6E73F8
:1075200020202020000072656C6163686572206213
:107530006F75746F6E20000020202020532E562E71
:107540005020212020202020000020617474656ECE
:107550007465206482627574202000007665727202
:107560002E206475206D69726F6972200000657845
:10757000706F736974696F6E000020636F6E747250
:1075800061737465204C4344202000002082636CAA
:10759000616972616765204C4344202000002082AD
:1075A000636C616972616765206D61782E200000EF
:1075B00020207282676C6572206865757265202074
:1075C000000020207282676C6572206461746520FF
:1075D00020200000202056444D20616B74696620F5
:1075E0003F20202000002020202020206E6F6E20D1
:1075F00020202020202000002020202020206F7527
:107600006920202020202020000020636F757075E5
:10761000726520616C696D2E2020000020202020E2
:107620006C6174697475646520202020000020203E
:10763000206C6F6E676974756465202020200000DF
:107640002066757365617520686F72616972652067
:107650000000207365636F6E64657300206482634D
:107660006C656E63657220202000207365636F6E09
:10767000646573200000206578706F736974696FAA
:107680006E0066696E2064752070726F6772616D3E
:107690006D650000617474656E7465006D61696E7E
:1076A000742E2000202056444D2020002020706C95
:1076B000616E20002020768272726F75696C6C8218
:1076C00020202020000020646576826572726F752C
:1076D000696C6C822020000020206D656E7520672B
:1076E000826E8272616C20200000202020666F6311
:1076F000616C697365722020202000002064826321
:107700006C656E6368656D656E74202000002020D6
:10771000202020706F736500656E74657220706F35
:10772000757220617272887400006D61696E746593
:107730006E697220656E7465720070686F746F2078
:10774000656E20636F757273200020202020827484
:1077500065696E6472652020202000002074656DCC
:107760007073207369648272616C20200000206550
:107770006666616365722070726F672E203F00003D
:107780002065666661636572206461746573203F7D
:107790000000656E7265672E2076616C6575727388
:1077A000203F00002020696E666F726D6174696F02
:1077B0006E73202000002070726F67732E20656644
:1077C0006661638273200000206461746573202009
:1077D000656666616382732000002020656E7265B5
:1077E000676973747282202020002062617474655E
:1077F00072696A206C656567202100002020415570
:10780000422077697373656C656E202000002062EA
:107810006174746572696A207A77616B2020000058
:107820002020626174746572696A204F4B202020A9
:107830000000202073746172742074696D65722079
:1078400020200000202074696D6572206B6C6161DE
:1078500072202020000020206D656E75206B696508
:107860007A656E2020200000206D656E75206F66A1
:1078700020656E746572202000002020696E73748C
:10788000656C6C696E67656E2020000070726F67B2
:1078900072616D6D612074696A64656E00002020FC
:1078A00074696A647374697070656E2020200000CA
:1078B0006175746F206F6E747370616E6E696E6740
:1078C000000074696A64206F6E747370616E6E6913
:1078D0006E6700006D616E2E206F6E747370616E46
:1078E0006E696E6700002020202066756E637469E3
:1078F00065732020202000002067656C696576652F
:1079000020746F657473202000002020206C6F733A
:107910006C6174656E20212020200000776163680F
:107920007420746F7420737461727420000073701B
:10793000696567656C6F706B6C617070656E000077
:1079400062656C69636874696E6700007061757A5E
:1079500065202020202000006265656C64656E2033
:1079600020200000204C43442068656C64657268E8
:107970006569642000006D61782E2068656C64651F
:1079800072686569642000002074696A6420696E09
:107990007374656C6C656E200000646174756D2095
:1079A000696E7374656C6C656E2000007370696538
:1079B00067656C206F706B6C6170203F0000202049
:1079C000202020206E65652020202020202000001F
:1079D000206D696E7574656E00002067656F677253
:1079E0002E20627265656474652000002020676542
:1079F0006F67722E206C656E677465200000202012
:107A0000202074696A647A6F6E652020202000004F
:107A1000636F727265637469652077616172646512
:107A20000000207365636F6E64656E00206F6E7476
:107A30007370616E6E696E672000207365636F6E90
:107A400064656E2000002062656C69636874696E0D
:107A50006700207061757A652020202020007072F8
:107A60006F6772616D6D612065696E6465200000ED
:107A700020776163687420002020206E752020002C
:107A80002020534F4B2020002020666F746F200071
:107A90006E696574207665726772656E64656C6484
:107AA000000020207665726772656E64656C6420E4
:107AB00020200000206E61617220686F6F66646D27
:107AC000656E75200000207363686572707374655D
:107AD0006C6C656E20200000207374617274206FDE
:107AE0006E747370616E2E2000002062656C696395
:107AF00068742E002073746F70206D657420656E3D
:107B0000746572200000656E74657220766173740E
:107B1000686F7564656E000020206F706E616D6522
:107B2000206C6F6F707420200000202075697473C2
:107B30006368616B656C656E2020000020207374A3
:107B4000657272656E74696A64202020000070722C
:107B50006F67722E2077697373656E20203F000077
:107B600074696A64737469702077697373656E3FB2
:107B70000000776161726465206F70736C61616E83
:107B8000203F0000202020696E666F726D6174696D
:107B90006520202000002070726F67722E206765BC
:107BA000776973742020000074696A647374697063
:107BB00020676577697374200000206F70676573B4
:107BC0006C6167656E202000626174746572696122
:107BD00020736361726963610000202020736F73FA
:107BE00074697669726520202020000062617474D7
:107BF00065726961206465626F6C65200000626176
:107C00007474657269612063617269636120000048
:107C1000696E697A69616C697A2E2074696D657222
:107C200000002074696D657220646973706F7374ED
:107C30006F20000020736365676C69657265206D55
:107C4000656E75200000207374616E646279207324
:107C50007461746F2020000020206D656E75206FA8
:107C600020656E7465722020000020202020207383
:107C70006574757020202020200070726F6772611B
:107C80006D6D612074656D706F20000020206F7233
:107C90006172692073636174746F20200000207327
:107CA000636174746F2070726F6772616D2E000073
:107CB00073636174746F2064692074656D706920EA
:107CC00000002073636174746F206D616E75616C68
:107CD000652000002020202066756E7A696F6E692D
:107CE000202020200000206C6173632E2070756CB2
:107CF00073616E74652000002020706572206661DB
:107D0000766F7265202120200000617370657474A5
:107D100061726520696E697A696F0000626C6F63D9
:107D2000636F20737065636368696F20000065731B
:107D3000706F73697A2E2020000070617573612066
:107D4000202020200000696D6D6167696E69202028
:107D5000000020636F6E74726173746F204C434433
:107D600020200000206C756D696E6F73697485202A
:107D70004C43442000006D61782E206C756D696E57
:107D80006F7369748520000020616767697573747B
:107D9000617265206F7261200000616767697573A9
:107DA0007461726520646174612000002020425378
:107DB0002061747469766F203F202020000020200D
:107DC00020202020206E6F20202020202000202036
:107DD0002020202020738D20202020202020000023
:107DE000206D696E75746920000067656F672E20CD
:107DF0006C617469747564696E65000067656F2EE7
:107E0000206C6F6E6769747564696E650000202070
:107E10006675736F206F726172696F202020000099
:107E2000202020636F7272657A696F6E6520202052
:107E30000000207365636F6E646920006F72617269
:107E4000692073636174746F2000207365636F6EC3
:107E5000646920200000206573706F73697A2E209A
:107E60002000207061757361202020202000707236
:107E70006F6772616D6D612066696E69746F000075
:107E8000617474657361200061646573736F2000B1
:107E90002020204253202000202020626C6F63634A
:107EA00061727369202020200000206E6F6E2062B6
:107EB0006C6F636361727369202000006D656E757D
:107EC000207072696E63697069616C650000206D75
:107ED0006573736120612066756F636F20200000F9
:107EE0007072656D69207065722073636174742EA1
:107EF00000006573706F73697A2E200020707265C0
:107F00006D69207065722073746F702000002020EE
:107F10007072656D6920656E746572202000206640
:107F20006F746F20696E20636F73736F2000202061
:107F30002020737065677565726520202020000021
:107F40002074656D706F207374656C6C6172652050
:107F50000000636F6E63656C6C6120706172616DAF
:107F60002E3F0000636F6E63656C6C61206F726101
:107F70007269203F000073616C7661206920706136
:107F800072616D2E203F00002020696E666F726D59
:107F90006174696F6E65202000007061722E20632D
:107FA000616E63656C6C6174692000006F72697248
:107FB000692063616E76656C6C6174690000207382
:0A7FC000616C7661746F20202000D0
:00000001FF
